:100000006F30704713000000130000001300000061
:100010001300000013000000130000001300000094
:100020001300000013000000130000001300000084
:08003000130000007300100032
:100038000000000000000000880200008C020000A0
:1000480000000000043C0000000000000000000068
:10005800063C0000083C0000000000000000000012
:100068000A3C0000000000000C3C000000000000FA
:100078000E3C0000103C0000123C0000143C000044
:10008800163C0000183C00001A3C00001C3C000014
:100098001E3C0000203C0000223C0000243C0000E4
:1000A800263C0000283C00002A3C00002C3C0000B4
:1000B8002E3C0000303C0000323C0000343C000084
:1000C800363C0000383C00003A3C00003C3C000054
:1000D8003E3C0000403C0000423C0000443C000024
:1000E800D8020000483C00004A3C00004C3C00009C
:1000F8004E3C0000503C0000523C0000543C0000C4
:10010800563C0000583C00005A3C00005C3C000093
:100118005E3C0000603C0000623C0000643C000063
:10012800663C0000D00200006A3C000000000000AD
:10013800000000006C3C0000723C0000743C0000B1
:100148006E3C0000703C0000000000000000000051
:100158000000000000000000000000000000000097
:100168000000000000000000000000000000000087
:0801780000000000000000007F
:10018000397101436EC619A0397141536AC866CAF4
:1001900062CC5ECE19A0397101535AD056D252D4D6
:1001A0004ED64AD826DA22DC06DE3301614082824E
:1001B00041114AC026C222C406C68282B24D410104
:1001C000024D924C224CB24B4101024B924A224AC0
:1001D000B2494101024992442244B2404101828025
:1001E0003D432A876373C3029377F700BDEFADE504
:1001F000937606FF3D8ABA960CC34CC30CC74CC716
:100200004107E36BD7FE11E28280B306C3408A0642
:100210009702000096966780A6002307B700A30602
:10022000B7002306B700A305B7002305B700A30452
:10023000B7002304B700A303B7002303B700A3024A
:10024000B7002302B700A301B7002301B700A30042
:10025000B7002300B700828093F5F50F93968500D1
:10026000D58D93960501D58D61B79396270097029A
:10027000000096968682E78086FA9680C1171D8FC9
:100280003E96E374C3F8A5B77300203037C500006D
:1002900013058594EFA0804AEF302044AA8537C526
:1002A00000001305C595EFA02035EF306043AA8507
:1002B00037C500001305C596EFA00034EF3080412C
:1002C000AA8537C500001305C597EFA0E03201A04D
:1002D000EF308021730020302945EF20F06C8545F8
:1002E00037050040EF30300073002030AA8519C573
:1002F00037C50000130585A26FA000308280011170
:100300008545054506CE02C202C423160100EF3022
:10031000E06E83A7418137470F0013070724B3D747
:10032000E7024C003705004023150100FD17231498
:10033000F10089679387F7703EC2EF30A06F0546E2
:10034000854537050040EF30A078854537050040EA
:10035000EF304076854537050040EF30C078F240F9
:10036000B7E700E0056723A2E710056182805D71B1
:100370001306C0038145480086C6A2C4A6C28D35B7
:1003800083D70181372400204C003ED6130504E8B2
:100390008D473ED0EF40A036834504E8AA8437C598
:1003A000000013058598EFA0202526858137034599
:1003B00004E8EF4090361D3FB64026449644616104
:1003C0008280797181454ECE06D622D426D24AD07B
:1003D00052CCAA8902C6EF40A0672AC235C5138451
:1003E00041860C4050004E85EF4060571C4012463D
:1003F000370A0020B2971CC09387018603D70700F5
:100400003714002034003A96420641829305843125
:1004100013054A192390C700EF10B00A9384418650
:100420001389018609CD50006C0013054A19EF109D
:10043000700511C5B24550004E85EF40900B130476
:1004400084312310090080C0B250225492540259C2
:10045000F249624A45618280411122C4056637141F
:10046000002013058431130686B69305F00F06C6E7
:10047000853B1304843123A281862244B240239019
:100480000186370500201305451941016F10207EB4
:10049000011122CC4AC806CE26CA4EC693F74500A3
:1004A0002A842E8991C3313F93778900B5CB854546
:1004B0002285EF4050210566130686B6B305C402B7
:1004C000B7270020938747E82285B7140020BE9500
:1004D000EF40C04303C744319307F00F9384443186
:1004E0006300F70C03C7140089496317F7008549B7
:1004F0008547A6972380870037C500001305059E12
:10050000EFA0C023CE9483C5040037C500001305B7
:10051000859FEFA0600EB7170140214723AAE7800F
:10052000937709018DCFB717002003C74731938711
:100530004731630A870603C717006317870005471B
:10054000BA977D572380E70037C50000130585A0C3
:10055000EFA0C01EB7170140214723A8E7801379F9
:10056000090463060904B717002003C747319387BE
:100570004731630C870203C71700631787000547DD
:10058000BA977D572380E7006244F240D244424943
:10059000B24937C50000130585A105616FA0001A97
:1005A00081498147B9B7014761BF0147D1BFF240D7
:1005B0006244D2444249B24905618280411122C459
:1005C00006C6EF40D00B937715002A8499C737C52C
:1005D00000001305059AEFA060169377240099C7D1
:1005E00037C500001305459BEFA0401593774400E5
:1005F00085C3EF40B00C11891DCD37C50000130530
:10060000C59CEFA0A013B7170140414723AAE7807C
:1006100041881DC80145EF40D007AA8519C1014591
:10062000853D0545EF40F006AA8519CD2244B2402C
:1006300005454101B1BDB7170140414723A8E780F7
:10064000214723A8E780E9B7B240224441018280D4
:100650000565011185451305C50306CE02C202C416
:1006600002C6EF30C037FD472312F10037150140B5
:100670008D473EC44C00C147130505803EC6EF3090
:10068000601CF24005618280797106D622D426D2A0
:100690004AD04ECE52CCEF3000055D3FB717014037
:1006A000094723A8E780054723AAE780114723AA23
:1006B000E780414723A8E7807165214723A8E780A9
:1006C00013050520EF30400B37C50000130585A347
:1006D000EFA0C00683A5418137C50000130585A49E
:1006E000EF909071EF30907BAA8537C5000013051D
:1006F00085A5EF907070EF30707AD1476308F500F0
:1007000037C50000130585A6EFA04003371400206D
:100710001305C430EF20102737C50000130585A747
:10072000EF90906D8144130AC430B7C90000194995
:10073000B387440183C50700138549A88504EF905A
:10074000B06BE39724FF2945EF90106F4D3E930661
:10075000C4301386C1809385418013858180EF204A
:10076000706E2A84613619E437C50000130585A828
:10077000EF90D07C9567938707E23EC2916793879D
:1007800087A93EC44800A5473EC6EF30D05DE93199
:10079000B71700207D57238AE73093874731A3801E
:1007A000E700F136EF20502FEF40806965DD3935E5
:1007B000D5BFB71702409843B706FFF8411113673A
:1007C000170098C3D84337060200758FD8C39843E3
:1007D000B706F7FEFD16758F98C39843B706FCFF62
:1007E000FD16758F98C3D843B70681FFFD16758F28
:1007F000D8C337079F0098C702C402C69843C16692
:10080000558F98C3B716024005679C42F18F3EC6CC
:10081000A24785073EC4B24781E7A247E397E7FEB8
:10082000B71702409C431397E700635707068547B5
:100830003EC632478547631FF704B7170240D843C7
:10084000B706C1FFFD16D8C3D843D8C3D843136732
:100850000740D8C3D843758FD8C3D843B7063500EF
:10086000558FD8C39843B7060001558F98C3984356
:1008700093166700E3DD06FED843B7160240719B6E
:10088000D8C3D84313672700D8C32147DC42B18BB4
:10089000E39EE7FE4101828002C661BFFD574165CC
:1008A0002380F50005058280FD5741652380F50012
:1008B00005058280597186D6A2D4A6D2CAD0CECEE2
:1008C000D2CCD6CADAC8DEC6E2C4E6C2EAC06EDE60
:1008D000834705007D4793C607086362D7027D3FC3
:1008E000B650265496540659F649664AD64A464B9F
:1008F000B64B264C964C064DF25D6561828013879F
:1009000007061377F70F9306E00563E4E600693FF7
:10091000C1BF138715003AC42380F5007547AE8424
:100920006374F7006F10A02C31678A07130707AABA
:10093000BA979C432A8982878347150011471385FC
:100940002500638AE7086362F70209476385E706C3
:10095000636BF70605476388E70401453704020027
:10096000A380A40009042295A5BF9306100F638DF0
:10097000D70663ECF6001307000FE390E7FE93073A
:1009800030032381F5000545D1BF9306E00F638B4B
:10099000D7069306F00FE392D7FC23810500A381CD
:1009A000E500094565BFB7C50000938585B1EF90A7
:1009B000B059254565B7B7C50000938545B2EF909E
:1009C000B058494561BFB7C50000938585B3EF9026
:1009D000B0572D4561B7B7C500001146938545B4A2
:1009E000EF90303611459DBF930700042381F50039
:1009F00093072004A381F500BD472382F500A3825D
:100A00000500CDB72381E500BDBF8347150089CF21
:100A10000547638BE700FD57A380F500370402000C
:100A200005044165050581B703472900B717014053
:100A300093870780058B11C70947D8CBA380040093
:100A4000F1BF094798CBDDBF8347150099CB054916
:100A50006389270109476380E7068147A380F40083
:100A600095A6B73700200547238AE754371401407D
:100A700091472328F440414923282441130404408A
:100A80000D474C1022853AD42312F1024AD6EF20AA
:100A9000705B4C10228523122103EF20B05A85474A
:100AA0001CC851474C1022852312F1023AD6EF2080
:100AB0007059854765B737370020230AF754371434
:100AC0000140B9472328F440C14923283441930702
:100AD0008004130404403ED64C10A1472285231203
:100AE000F102EF2030568D473ED44C1099472285B5
:100AF0002312F1024ED6EF20F0544C10228523121F
:100B00003103EF203054D147232824014C10228593
:100B10003ED623122103EF20F052894781B7B73721
:100B2000002037140140238A0754B94713050440B5
:100B30002312F1024C1091473ED6EF20B050C1472E
:100B4000130504404C102312F102EF20B04F8547EB
:100B5000130504404C102312F1020544EF20904E7F
:100B6000A38004007DBD8347290003451500A2072B
:100B70005D8DEF20B039D9B53714014005492328E0
:100B8000244113052003EF20D03B232A2441238155
:100B90000400A3800400094469B503474500834766
:100BA00035008345250022075D8F8347550013F3E9
:100BB000150003461500C2075D8F83476500E207F5
:100BC000D98F630C03003717014093761600130783
:100BD0000740638D0610914614CB13FE2500630C6D
:100BE0000E003717014093762600130707406382F3
:100BF0000610C14614CB93FE4500638C0E0093563D
:100C0000260037170140858A13070740F5C6894635
:100C100014CB939F850193DF8F4163DB0F00371760
:100C200001409356760013070740F1CA854654CB1E
:100C3000BDCF37C72D001307076C6373F700BA8762
:100C400013858186032805009352160093532600CE
:100C50001307180018C11354560013597600014F9A
:100C60009386818693F50502B71801401348F8FF73
:100C70006308030003A58840098105896319A60854
:100C800063080E0003A58840118105896391A208BD
:100C900063880E0003A58840058105896399A30632
:100CA00091C135E463C00F0663030F0098C2371784
:100CB000014083268740832787400326874083257A
:100CC00087408D831307074006061847898B118AD2
:100CD0008982858AD18FD58F93F68500D58F1E079F
:100CE000D98FA380F400370406001DBB914654CB76
:100CF000EDB5C14654CB01B7894654CB19BF8546E3
:100D000014CB3DB703A588400589E30FA9F8050773
:100D10003305E800054FE36DF5F449BF03472500AF
:100D20008347150022075D8F83473500C2075D8F1B
:100D300083474500E207D98F99E7FD57A380F50067
:100D400037040400F1B9856637370020938686386A
:100D500013074755639AD7008547A300F7008547D7
:100D60005CC3A3800400E9BF83A641812946A30098
:100D70000700B3D6C602B3D7F602DDB703441500A9
:100D80009305250019E01304001022851D04EF10BF
:100D9000503B0D80A380040005044204136414003A
:100DA00049B183471500373700201307475593F69D
:100DB000370089838506858B230CD700A30CF700A9
:100DC000A38005004164A9B9A3800500034A15006A
:100DD000B709F1FF1384250093072500054B8544CF
:100DE000FD5CB70B0020FD19370C0300370D040024
:100DF0007D1A63179A01139404013364640115B1D9
:100E000003C50700938A17001379F50363140900DB
:100E10001309000403A70B07931D85011D091C433B
:100E200093DD8D4113593900B3F7370163DA0D02B1
:100E3000B3E7A7011CC32286D685EF101039631AC9
:100E40000A0003A70B071C43B3F73701B3E7870179
:100E50001CC3850463D90D004A944A9BD68749BFB9
:100E6000B3E78701C1BFCA9ACA94CDBFA38005006A
:100E700003441500938A250093072500054A8544FD
:100E8000FD5B7D1463177401139404013364440102
:100E900049BE83C90700138B170013F9F9036314C4
:100EA0000900130900044E851D095686DA85135979
:100EB0003900EF00B06CE2091307190093D989419A
:100EC000B3072B01BA94E3DE09FACA9A4A9A55BFCE
:100ED00003441500B737002013874755230D8700BB
:100EE0009386475593854755014693874755014754
:100EF00085078905636B8600368681478506090666
:100F000063E08702A380040041BD3305C9000345A7
:100F100025000506A38DA7002391E5022A97C9BFE6
:100F200083C5B60185070D8F2319E602C1BFB73708
:100F3000002083C6475509476393E604034715001D
:100F400093874755A38DE70083C7A7016379F7020D
:100F50003945EF10201AEF00306E9357850023813A
:100F6000A400A381F4004164935705016181A3802B
:100F700004002382F400A382A40015045DB4FD578D
:100F8000F1BC03471500B7370020938747552386E8
:100F9000E70003473500834625002207558F239835
:100FA000E70003475500834645002207558F2399E4
:100FB000E700A3800400370405009DB493071500E3
:100FC000B73900203ECA83C749553EC632478547D8
:100FD0006305F70289476302F746034725001304B8
:100FE0003500E3170704D247A380040023810400DF
:100FF0001D8C4204136424002DB4B7360020B7378B
:101000000020130D3500834B2500938D3500238C74
:101010000658014A014B014502C83689938C475551
:10102000894A8549639B0B0485466319D502630E83
:101030000B3CB7370020138B475583590B01094AE6
:101040004C103945EF103025631E4539638809007F
:1010500003478959FD191377F70F7DD3C2472381C1
:10106000A400A380F400D247B307FD401395070105
:10107000A2473384FD40498C6DB203440D009307B1
:101080001D003EC693752400638F052663010B0C7B
:101090009375140103DC0C01639F35034C1022850A
:1010A000EF10701F631A550563080C0083458959BA
:1010B0007D1C93F5F50FFDD1324D83460D0013F6DF
:1010C0002600630F0630C18A639C0630050DFD1BA8
:1010D000E3950BFE91BF4C103945EF10D01B631CFC
:1010E000550163080C00034789597D1C1377F70FDE
:1010F0007DD3014BD1B7014BE31035FD925513D889
:1011000085002380BD00A3800D0113D80501E18176
:1011100023810D01A381BD0013884D0063090B08D5
:1011200093158401E1855A8563D3050883A58C0056
:10113000A10D13D58500238EBDFEA38EADFE13D564
:101140000501E181238FADFEA38FBDFE5A85937506
:10115000040103D80C0113731400F1C183452D0061
:10116000034C1D0093075D00A205B3E58501034C08
:101170003D003EC6420CB365BC00034C4D0003DD90
:101180002C01620C336CBC0063070302814522858D
:1011900042CCEF105010631E55016248E30E08F078
:1011A000834789597D1893F7F70FEDD331B7C28D77
:1011B00079BFE31335F103D80C014C10228542CCE2
:1011C000EF10700DAA876316550362486308080084
:1011D000834589597D1893F5F50FE5D183A64C0118
:1011E0009255ED8E6309DC0213E507011375F50FC7
:1011F000E1B503A84C019255B3F50501E31035FFA5
:10120000E30EBCFCE30C0DFC834589597D1D93F571
:10121000F50FD5D1E1B7E39137EB014AB9A8630CDB
:101220000306E31C0BFE8145228542CCEF10B0067D
:10123000631C55016248E30E08EA834789597D180B
:1012400093F7F70FEDD38DBDE31835E793168401BF
:10125000E18663D4061883A78C00014A054B13D797
:1012600087002380FD00A380ED0013D70701E183F1
:101270002381ED00A381FD00910DC2479386FBFF02
:1012800085073EC88347895993F7F70FE39607E22E
:10129000B68B324D41BB4C10228542CCEF10A07F63
:1012A000631C55016248E30908E0834789597D18AA
:1012B00093F7F70FEDD309B5E31035E193168401E9
:1012C000E18663D2060283A78C00910D93D6870036
:1012D000238EFDFEA38EDDFE93D60701E183238FCF
:1012E000DDFEA38FFDFE9257910D93D68700238ECE
:1012F000FDFEA38EDDFE93D60701E183238FDDFE85
:10130000A38FFDFE19BF63040B0403DC0C014C101A
:101310003945EF104078631B5501E30F0CD8834526
:1013200089597D1C93F5F50FFDD179B3E31635D9B5
:101330001257910D93558700238EEDFEA38EBDFEAF
:10134000935507016183238FBDFEA38FEDFE834577
:101350002D0003471D0093075D00A205D98D0347AB
:101360003D003EC6937704024207D98D03474D00E6
:1013700062074D8F3AD291C723AAEC00014B054575
:10138000EDBD03DB0C014C102285EF10C070631B18
:101390005501E3030BD2834789597D1B93F7F70F60
:1013A000FDD381BBE31735D593168401E186054A49
:1013B00063D3060283A78C00054A910D13D78700DB
:1013C000238EFDFEA38EEDFE13D70701E183238F4D
:1013D000EDFEA38FFDFE014B4DB5014A054B71BDDE
:1013E000150DF5B10547E31BE5C61257910D935650
:1013F0008700238EEDFEA38EDDFE935607016183E9
:10140000238FDDFEA38FEDFE91B9E3090AC4B73740
:101410000020138B475583590B01094A81453945F3
:10142000EF106067E31C45C3E38A09C2034789598B
:10143000FD191377F70F7DD315B103471500938678
:101440004955B73A0020A38DE60083C6A601238C38
:101450000A58938C3500938949556376D73C130D10
:101460003500034C25000146814D01450144094BDF
:10147000854B631C0C0432890546631BC502294653
:101480006305C9002945EF00F04603D909018949E0
:10149000638C0D364C103945EF00906F6313353572
:1014A0006308090083C68A597D1993F6F60FFDD2A9
:1014B000D247A38084002381A4003307FD40A247C4
:1014C000131507013384FC407DB6034A0D009307D2
:1014D0001D003EC813791A0093752A0029096388F4
:1014E000052263840D0C03D8090163192603937543
:1014F0000A018DE54C10528532CE42CCEF00506986
:1015000072466319650562486308080083C58A59F5
:101510007D1893F5F50FF9DD3289FDA0A947630722
:10152000F600294542CCEF00F03C6248C28D4C10D9
:101530003945EF00F065631D650163840D2003C626
:101540008A59FD1D1376F60F7DD22949814D6DA86C
:101550002946814DE31275FD925513D885002380ED
:10156000BC00A3800C0113D80501E18123810C018B
:10157000A381BC0013884C0063870D0A93158A0170
:10158000E1856E8563D1050A83A58900A10C13D579
:101590008500238EBCFEA38EACFE13D50501E18130
:1015A000238FACFEA38FBCFE6E8593750A01638FFB
:1015B000050E83452D0003451D00A2054D8D834575
:1015C0003D00C205C98D03454D006205B367B500F6
:1015D0003ECC93075D003EC803DD29016305C900C9
:1015E0004A85EF00303103D609018145528532CE5C
:1015F000EF00105A631B6503724619C603C78A5968
:101600007D161377F70F75D3424D03460D00937582
:1016100026006386051C418A6313061C050D7D1C8C
:10162000E3150CFE91BDC28C49B7E31F75FD03D6CF
:1016300009014C10528532CEEF0090552A87631C69
:101640006501724619C603C78A597D161377F70FCD
:101650006DD3324715A003A6490192556D8E631DC7
:101660007501E247638AC70063080D0003C68A5903
:101670007D1D1376F60F45DE03A649019255E2471C
:101680006D8E6387C700136507011375F50FADBF36
:10169000E31C75F703C78A5905049305FCFF13770C
:1016A000F70F3DF34A862E8C424DE1B363970D123E
:1016B0006305C9004A85EF00F02303DD0901814578
:1016C0005285EF00F04C631B6501E3010DE803C791
:1016D0008A597D1D1377F70F7DD33DB7E31675F358
:1016E000620A135A8A41854DE3560AFA03A7890014
:1016F000910C13568700238EECFEA38ECCFE13565E
:1017000007016183238FCCFEA38FECFE61B7638E4C
:101710000D04A9476305F6002945EF00B01D03D865
:1017200009014C10394542CCEF009046631D65011C
:1017300062486308080003C68A597D181376F60FBD
:101740006DD22949D1B5E31E75FF9256910C13D67F
:101750008600238EDCFEA38ECCFE13D60601E1822A
:10176000238FCCFEA38FDCFE294683452D008346C4
:101770001D0093075D00A205D58D83463D003EC840
:1017800013770A02C206D58D83464D00E206CD8E40
:1017900036D219C723AAD9003289814D0545DDBD4E
:1017A0006305C9004A85EF00F01483DD09014C1080
:1017B0005285EF00F03D631B6501E3870DE403C72D
:1017C0008A59FD1D1377F70F7DD349B3E31075D9FF
:1017D000620A135A8A41814D01BF328965BD150DD8
:1017E0003DBD8546E316D5CC9256910C13D68600A6
:1017F000238EDCFEA38ECCFE13D60601E182238F5E
:10180000CCFEA38FDCFE6DB181453945EF00503829
:10181000E31035CBE30E09C883C68A597D1993F6C8
:10182000F60FFDD271B1130D25000144014549B1F8
:101830008347040093F6270099C6C18B89E7050406
:101840007D176FF00FFA1504E5BFB739002083C785
:1018500049550547638DE7000947638DE716A38067
:10186000050023810500A38105000D446DA0834A76
:10187000350083472500373C0020A20A230C0C5872
:10188000B3EAFA00938C450063840A14034D4500C3
:101890009389495593772D0095EB930B5500014A99
:1018A000894D03DB090163914A0F8949FD5A81453E
:1018B0003945EF10401E631535057D1B63025B053E
:1018C00083478C5993F7F70FFDD31DA893771D001D
:1018D000C5CB03DA0901094B81456A85EF10A01BCE
:1018E000631C6501630E0A0083478C597D1A93F7C8
:1018F000F70FFDD3014A29A08547014A6302F50885
:10190000A247A3804401135A8A0023814401A38182
:10191000A4003384FC4083474900898B638E0722EF
:10192000370504006FF02FF5FD1AE31B75FD925784
:10193000910C050A13D78700A38EECFE13D707017D
:10194000238EFCFE238FECFEE183A38FFCFEE38954
:101950000AFA63967A0193771D0091C3394D03DB30
:1019600009014C106A85EF100013E31FB5FBE30972
:101970000BF883478C597D1B93F7F70FFDD349B7BD
:10198000014A854B894DF1B703C71B0083C70B0084
:10199000910B22075D8F83C7EBFFC2075D8F83C763
:1019A000FBFFE207D98F3ED24C106A85EF10A00EE4
:1019B0008546631BB501E3050BF483478C597D1BFA
:1019C00093F7F70FF5D32DBFE31CD5F2050AD1BD70
:1019D00001450DB78347150013874955373B002054
:1019E000A30DF7000347A701230C0B58938A45006A
:1019F0009389495563F0E716034A3500834725006C
:101A0000220A336AFA0063070A14834C450093FBE9
:101A10001C00A90B5E85EF00E06D93F72C00668C2F
:101A2000A1EB130C5900814D094D054483461C0060
:101A300003470C00110CA206D98E0347ECFF4207A6
:101A4000D98E0347FCFF6207558F83D609013AD22E
:101A50004C10668536C6EF00B0136310A50DB24674
:101A6000BDCA03478B59FD161377F70F75D3A5A091
:101A700083DD0901094D81456685EF007011631C06
:101A8000A501638A0D0403478B59FD1D1377F70FDA
:101A90007DD3814D89A00547814D631EE502854CAC
:101AA0002944094D63189A01394C63858B002945F7
:101AB000EF00406483D609014C10628536C6EF0002
:101AC000300D6316A503B24699C603478B59FD1620
:101AD0001377F70F75D393D78D002381F400A247B6
:101AE000A380B401A381A4003384FA402DB57D1AEC
:101AF000E31395FF1257910A850D93568700A38E25
:101B0000DAFE93560701238EEAFE238FDAFE618305
:101B1000A38FEAFEE3180AF87DBFE31E85FA850D60
:101B2000E316BAF129476385EB002945EF00805C95
:101B300083D90901094A81453945EF007005E31C45
:101B400045F9E38A09F803478B59FD191377F70F15
:101B50007DD351B7014535BF03453900834729007F
:101B600022055D8D05054A056FF0EFD0B7370020DF
:101B700003C747558546630AD7008946630CD702D9
:101B8000FD57A380F4006FF00FC303473500834770
:101B900025004C1022075D8F83474500C2075D8FEB
:101BA000834755000145E207D98F3ED2EF00B06E62
:101BB0006FF02FC00347150093874755A38DE700AB
:101BC00083C7A701E37EF7FA21452D23034539009A
:101BD0008347290022055D8D83474900C207C98FCD
:101BE0000345590062055D8DA5266FF08FBCFD573A
:101BF00041652380F40005056FE09FCE8346050014
:101C00001306F0076393C606011122CC4AC84EC6DC
:101C100052C456C206CE26CA2380D500834415007E
:101C200037040200416A1309250093892500A38027
:101C300095000904FD5A7D1AFD14639C5401228508
:101C4000F2406244D2444249B249224A924A056172
:101C50008280CE854A85EFE0FFC5935705012A941F
:101C6000337545013E99AA99C1BF6FE0BFC485672E
:101C70003E95914723280500232A05001CC52326ED
:101C8000050082808567B306F500D8460DCB7D1729
:101C9000D8C6D84A93870780BA978607AA9783D76A
:101CA00007001318A7002A9823A005011CC29C4610
:101CB00005070D8B8507D8CA9CC60545828001455E
:101CC00082808567AA97984749C3011122CC06CE26
:101CD00026CA4AC84EC652C47D1798C79C4B2A8450
:101CE000AA073E959307004063D4C700130600403F
:101CF000856433099400368AAE89EF809004832589
:101D000009014E8593840480AA05A295C53D8327C9
:101D10000901F240B249BE948604A2942390A40023
:101D20001395A7002A94850723208A008D8B2328EA
:101D3000F9008327C9006244D24485072326F900AD
:101D4000224A424905450561828001458280B717D4
:101D50000140058993870740094719C198CB8280C4
:101D6000D8CB8280B717014003A587400D81058934
:101D700082807D1511E182800100E5BF397126DA8C
:101D800006DE22DC4AD84ED652D456D25AD05ECE87
:101D900062CC66CA9374F50399E093040004B71704
:101DA0000140137705049387074041C7414798CB0B
:101DB000B7390020371B0140914A9389495513795F
:101DC0000508850583CBF5FF214A014495CC13F521
:101DD000FB0F32C62EC4A53F232A5B4103A5490051
:101DE00005807D1A7937BD3F23285B412A8C03A5E6
:101DF00049001E0C93DB1B00AD3F33648C00FD14C7
:101E0000A2453246E3140AFC630709003354440137
:101E1000230086000506D5F4F2506254D25442598C
:101E2000B259225A925A025BF24B624CD24C216157
:101E300082804147D8CBADBF011106CE22CC26CA45
:101E40004AC8B71401404EC652C456C25AC0414A8D
:101E5000914923A84441373400201309445523AA4B
:101E600034410325490013044455213723A8344144
:101E700003254900FD3D23AA444123AA34410325FB
:101E80004900371A0140F53523A83441032549009C
:101E9000CD3523AA344103254900E13D23A834412F
:101EA000032549009144F1350349B90148406318BD
:101EB0000908B71401407D4A938404409149114BAD
:101EC00023AA640148407D1A6D35693D23A8340179
:101ED000AA8A4840FE0A33E92A01613D13591900D4
:101EE000E3100AFEC14A23A8540123AA3401484042
:101EF00049358D3D23A834012A8A48407E0A33693A
:101F00002A01853D23AA34014840A53523A8340180
:101F10004840853523AA540123AA34014840913D05
:101F200023A834014840B135F24062444A85D24486
:101F30004249B249224A924A024B05618280232AD1
:101F40009A40053D23289A4048407D191D35B9BF68
:101F5000011106CE22CC26CA4AC8B71401404EC68B
:101F600052C456C2C14A114A23A8544137340020F2
:101F70001309445523AA4441AA890325490013049F
:101F80004455C53B23A8444103254900DD3323AA1A
:101F9000544123AA444103254900B71A0140D13BCB
:101FA00023A8444103254900E93323AA44410325DA
:101FB0004900C13323A84441032549005D3B03493F
:101FC000B901484093840A406319090E8947DCC867
:101FD000114923AA2401713B23A824014840B71AC0
:101FE0000140114A793323AA24014840593323A8D8
:101FF00024014840BD3B23AA240148409D3B23A81F
:1020000024014840FD44B53313F5F90F13890A4004
:102010003D3B232A49014840FD1493D91900913BC7
:10202000232849014840B133E5F08347B401834494
:10203000A40113F5F90F9D8C85476382F40A013BD7
:10204000232A49014840F91491492533232849019D
:102050004840371A0140313B484013090A40BDE46B
:10206000C1472328F9009144232A990019332328D2
:1020700099004840B71401401149E53923AA244189
:102080004840C53923A824414840E531C14723AA27
:10209000F44023AA24414840E93923A82441484078
:1020A000C939F2406244894723A8F4404249D244E6
:1020B000B249224A924A0561828023AA44015539D5
:1020C00023A8440148407D196D31E5BD232A39011B
:1020D0004D31232839014840FD146139B5BFC1474E
:1020E0002328F900AD31232A4901484059312328DA
:1020F000490141B7011122CC3734002026CA4EC60F
:102100009307445506CE4AC852C456C283C7170027
:10211000B7140140AA891304445593840440FDC7B1
:10212000414798C89147DCC89CC8DCC89CC8D8C83F
:10213000DCC89CC8DCC89CC889479CC80347B4015C
:10214000B71501409146930787008607A29783D76A
:102150004701D9E322978344C701371A0140114947
:10216000FD1413F5F90FBDEC8347B401C1078607D1
:102170003E94835444013714014013040440BDCC01
:10218000F93691475CC81CC889471CC8B71601407E
:102190001147FD1493870640B9EC414798CB11478E
:1021A000D8CB98CBB7170140114723AAE74023A803
:1021B000E740C14623AAD74023AAE74023A8E74027
:1021C000094723A8E740F2406244D2444249B24959
:1021D000224A924A0561828023AAD54023A8D5408D
:1021E000FD1785BFEFF0BFB6232A2A4123282A41D5
:1021F00093D91900B5B7D8CB98CB61BFC1471CC8DC
:10220000EFF0FFB491475CC81CC869BF414A11494F
:1022100023A8440123AA24014840B71A0140EFF043
:102220005FB523A824014840EFF0BFB423AA2401DE
:102230004840EFF01FB423A824014840EFF07FB3DB
:1022400023AA440123AA24014840EFF09FB223A807
:1022500024014840EFF0FFB123AA24014840EFF0E9
:102260005FB123A824014840EFF0BFB089479CC864
:102270008347B401A1078607A29783D44701DDE80D
:102280008347B401B71A01401149A29783C4C7011B
:10229000FD1413F5F90FDDE88347B401B7140140CD
:1022A00093840440C1078607A29703D947016308B6
:1022B000090C9149EFF0BFA923AA34014840371A0D
:1022C0000140EFF01FAB23A834014840EFF07FAA94
:1022D00089479CC87D19484093040A406317090840
:1022E000C1479CC8114923AA2401EFF09FA823A845
:1022F00024014840B71401401149EFF09FA723AAD9
:1023000024414840EFF0FFA623A824414840EFF0C5
:102310005FA6C14723AAF44023AA24414840EFF016
:102320005FA523A824414840EFF0BFA4894723A814
:10233000F44051BD23AA2A414840FD14EFF07FA389
:1023400023A82A414840EFF0DFA215BFEFF03FA0DD
:1023500023AA2A41484093D91900EFF09FA123A84E
:102360002A414840EFF0FFA025B723AA3401EFF03F
:102370005FA023A834014840EFF0BF9FA1BFC14731
:102380009CC81149EFF0BF9C23AA24014840B1BF6B
:10239000797122D43734002026D24AD052CC930708
:1023A000445506D64ECE56CA5AC85EC662C466C2E8
:1023B00083C71700B71401402A892E8A1304445595
:1023C0009384044063810722414798C89147DCC841
:1023D0009CC8D8C8DCC89CC8DCC89CC8034BB401E6
:1023E000B716014063100B0EB714014013551900C6
:1023F00093840440914A1375F50FEFF05F9523AA7B
:102400005401EFF03F96AA8B135529001375F50F71
:1024100023A85401EFF0BF9323AA5401EFF09F9437
:10242000AA89135539001375F50F23A85401EFF04D
:102430001F9223AA5401EFF0FF92860B0A05B3EB1B
:10244000AB0023A85401B3E9790185476382F908F9
:10245000C1479CC823AA540123A85401B7170140BF
:10246000114723AAE74023A8E740C14623AAD74043
:1024700023AAE74023A8E740094723A8E7401379A8
:102480000908630909009387C186984393061700DA
:1024900094C318C48347C4007D56B7150140114743
:1024A000FD17639DC712B250225413F5F90F9254D1
:1024B0000259F249624AD24A424BB24B224C924CE8
:1024C0004561828023AAF64023A8F6407D1B19BFF0
:1024D00093772900D9C3FD4A914B114C23AA84015B
:1024E000EFF05F887E05336B650123A87401FD1A48
:1024F000135B1B00E3940AFE8347A401834AB401E3
:10250000B38A574185476381FA0423AA7401EFF027
:102510007F859387EAFF23A874013716014091460F
:102520001307064091EFC1471CCB91475CCB1CCBF6
:10253000E3060AF27E05336B650123206A0139BF89
:1025400054CB14CBFD17E9BFC1479CC823AA740123
:10255000EFF05F8123A87401E1BF832A0A00FD44E4
:10256000B71B0140114B13F5FA0F138A0B40EFF024
:102570000FFE232A6A0123286A01FD1493DA1A0048
:10258000FDF08347A4018344B40113F5FA0FB3842B
:1025900097408547638AF402EFF06FFB232A6A01B4
:1025A00023286A019387E4FF3716014091461307F9
:1025B000064099E7C1471CCB91475CCB1CCB79BD4A
:1025C00054CB14CBFD17E5B7C1472328FA00EFF031
:1025D0000FF8232A6A0123286A0149B523AAE54096
:1025E00023A8E54075BDC14A914923A8540123AAF7
:1025F00034014840EFF0EFF723A834014840EFF0F2
:102600004FF723AA540123AA34014840B71A0140C6
:10261000EFF02FF623A834014840EFF08FF523AAFE
:1026200034014840EFF0EFF423A8340148409144CE
:10263000EFF02FF4834BB40163970B0AB7140140FA
:102640001355190093840440914A1375F50FEFF068
:102650000FF023AA54014840EFF0AFF1EFF08FF0F4
:1026600023A854012A8B4840060BEFF08FF0135536
:1026700029001375F50FEFF08FED23AA54014840A0
:10268000EFF02FEFEFF00FEE23A85401AA89484096
:10269000EFF02FEE135539001375F50FEFF02FEB18
:1026A00023AA54014840EFF0CFECEFF0AFEB23A8A2
:1026B00054012A8C4840EFF0CFEB13152C00336502
:1026C000AB00B3E9A9008547638BF902C1479CC8F9
:1026D00023AA54014840EFF0CFE923A85401484011
:1026E000EFF02FE965A823AA9A404840FD1BEFF0C0
:1026F0004FE823A89A404840EFF0AFE735BF937703
:10270000290063800714FD4A114C914C23AA9401BF
:102710004840FD1AEFF0EFE5EFF0CFE423A8840185
:102720002A8B48407E0B336B7B01EFF08FE4935B89
:102730001B00E39D0AFC8347B401834AA40148407F
:10274000B38AFA4085476382FA0E23AA8401EFF028
:102750004FE2EFF02FE123A884012A8B48409384B5
:10276000EAFFB71C0140EFF0CFE0114C4840938ADC
:102770000C40CDE0C14723A8FA00914423AA9A0057
:10278000EFF02FDF23A89A004840EFF08FDE6307B9
:102790000A007E0B336B7B0123206A01B7140140D2
:1027A000114A23AA4441484013790908EFF06FDC2D
:1027B00023A844414840EFF0CFDBC14723AAF440AF
:1027C00023AA44414840EFF0CFDA23A844414840CF
:1027D000EFF02FDA894723A8F440630909009387B3
:1027E000C18698439306170094C318C48344C40059
:1027F000FD5A371B01401149FD14E38654CB232AAF
:102800002B414840EFF0EFD623282B414840EFF012
:102810004FD6DDB723AA8A01EFF0AFD523A88A01EE
:102820004840FD14EFF0EFD491B7C1479CC823AAEC
:102830008401EFF00FD4EFF0EFD22A8B23A88401AC
:10284000A1B7832A0A00FD44B71B0140114B13F5C1
:10285000FA0F138A0B40EFF08FCF232A6A0148400A
:10286000FD1493DA1A00EFF0CFD023286A01484014
:10287000EFF02FD0E9FC8347B4018344A40113F5A2
:10288000FA0F9D8C8547638CF404EFF04FCC232A1C
:102890006A014840F914914AEFF0AFCD23286A014C
:1028A0004840371B0140EFF0CFCC4840130A0B40A3
:1028B00081ECC1472328FA009144232A9A00EFF0C3
:1028C0004FCB23289A0021BD232A5A01EFF06FCA6B
:1028D00023285A014840FD14EFF0AFC9F9B7C147AA
:1028E0002328FA00EFF0AFC6232A6A014840EFF030
:1028F0004FC823286A01E5B3B717014003A58740F5
:10290000118105898280B7170140058993870740A7
:10291000414719C198CB8280D8CB8280B70700206D
:1029200083A607073707F1FF7D179C42F98F37070A
:102930000300D98F9CC282807D1511E18280010045
:10294000E5BF39714AD83739002022DC26DA4ED665
:1029500052D456D25AD062CC06DE5ECEAA898144C9
:1029600001447D5C371A0140C14A114B1309495596
:10297000FD19639E8901F2506254D2544259B259F2
:10298000225A925A025BF24B624C2161828089E4A6
:1029900003C40500A14485059377140013070A407A
:1029A00095C3232857012EC6232A6A4103254900CF
:1029B0000580FD14513723286A4103254900AD3FA6
:1029C000B2457DB7232A5701F9BF397122DC06DEF3
:1029D00026DA4AD84ED652D456D25AD05ECE137486
:1029E000F50319E0130400041375050819C9B73974
:1029F0000020B71B0140914A9389495521498144E0
:102A0000BDA0B7340020B71A0140914993844455C2
:102A100003C90500130B84FF85051375F90F2EC636
:102A2000DD3523AA3A41C8407D14135919002937CE
:102A300023A83A41C8400937B245630C640571FCCC
:102A400035A832C623AA5B4103A5490085807D19BC
:102A5000E5355D3523A85B412A8A03A549001E0A96
:102A6000B3649A00D13D7D1432466303090071F8C6
:102A70000506B3D42401A30F96FE49F0F250625428
:102A8000D2544259B259225A925A025BF24B2161F6
:102A900082803DFCE5B7397122DC52D49357250082
:102AA000135A15003734002026DA4AD84ED656D2AB
:102AB0005AD05ECE62CC66CA6AC86EC606DEB7144D
:102AC0000140137CFA0F93FBF70F3E9A930744558E
:102AD00083C7170093840440C14C135735002A9ACA
:102AE00023A8940111493A9A23AA2401AA89AE8AFB
:102AF000937DF50F137BF70F137AFA0F13044455E8
:102B0000370D0020638D07266E8523A82401E53B41
:102B100023AA2401628523A82401F53323AA2401D2
:102B20005E8523A82401C53323AA24015A8523A83E
:102B30002401D13B23AA2401528523A82401E13397
:102B400023AA240123A8240123AA940123AA24014F
:102B500023A8240123A8940183260D0723AA240176
:102B600023A824019C423707F1FF7D17F98F37070F
:102B70000400D98F9CC2034A840137170140914752
:102B80001309074063100A0E114B232A6901AD3364
:102B900023286901232A6901AA84B93B23286901F2
:102BA000232A6901AA8BEFF03FD5860B0A05B3EB08
:102BB000AB0023286901B3E49B0085476399F412B5
:102BC00093F72900C5CF014B130C0002914B914C98
:102BD000232A9901EFF05FD22A9A135B1B007E052E
:102BE000232879017D1C336B6501E3130CFE232A36
:102BF0007901EFF07FD0334545012328790105891C
:102C000011C1A14463840A0023A06A01834784019F
:102C1000371601401147A9EFEFF05FD093F909088B
:102C2000638909009387018798439306170094C32B
:102C300018C40347C40045E3B7170140414723A820
:102C4000E740F250625413F5F40F4259D254B2598E
:102C5000225A925A025BF24B624CD24C424DB24D18
:102C600021618280232AF9002328F9007D1A09BFF7
:102C7000232AE6402328E640FD1771BF034984015B
:102C8000B7160140914763120904EFF03FC9930B57
:102C9000000203AB0A00371C0140914A1375FB0F79
:102CA000EFF07FC6232A5C4123285C41FD1B5A9923
:102CB000135B1B00E3940BFE1375F90FEFF0BFC419
:102CC000232A5C4123285C4191BF23AAF64023A814
:102CD000F6407D194DBFB7170140C14693870740A5
:102CE000D4CB9146D4CB94CB7D176DFFB1B713876E
:102CF000E4FF759B834784010DC311479306F0FDE4
:102D0000232AE9002328E900FD17E39BD7FEEFF013
:102D1000FFC0C1472328F9002DB7034794010DEFE9
:102D2000371601401147B1E7EFF05FBF83479401C9
:102D3000E38407F093F92900E39009F0B717014005
:102D4000414793870740D8CB914613071002D4CB55
:102D500094CB7D176DFFCDB513F7290071D3130701
:102D600010029146232AD9002328D9007D177DFB24
:102D700045BF232AE6402328E640FD176DB74840AB
:102D8000EFF09FBB23A824014840EFF0FFBA6E8507
:102D9000EFF07FB723AA24014840EFF0FFB923A842
:102DA00024014840EFF05FB96285EFF0DFB523AA58
:102DB00024014840EFF05FB823A824014840EFF019
:102DC000BFB75E85EFF03FB423AA24014840EFF07F
:102DD000BFB623A824014840EFF01FB65A85EFF094
:102DE0009FB223AA24014840371B0140EFF0DFB413
:102DF00023A824014840EFF03FB45285EFF0BFB064
:102E000023AA24014840EFF03FB323A824014840FF
:102E1000EFF09FB223AA940123AA24014840EFF0C7
:102E2000BFB123A824014840EFF01FB123A89401AB
:102E300023AA24014840EFF03FB023A824014840D2
:102E40009144EFF07FAF83260D073707F1FF7D1721
:102E50009C42F98F37070400D98F9CC2034A840132
:102E6000484013090B4063180A12114B232A6901C9
:102E7000EFF09FACEFF05FA823286901AA8C4840CF
:102E8000EFF09FAB232A69014840EFF0FFAAEFF073
:102E9000BFA623286901AA8448408604EFF0DFA971
:102EA000232A69014840EFF03FA9EFF0FFA423284F
:102EB00069012A8C48400A0CB3E48401EFF0DFA7D3
:102EC000B3E494018547639EF41693F72900638B5E
:102ED000070E014B930C0002114C114D232AA9013E
:102EE0004840135B1B00FD1CEFF01FA5EFF0DFA0B7
:102EF00023288901AA8B48405E9AFE0BEFF0DFA3DE
:102F000033EB6B01E39C0CFC232A89014840EFF072
:102F1000BFA2EFF07F9E23288901AA8B484033CAC5
:102F20004B01137A1A00EFF03FA163030A00A1449A
:102F300063840A0023A06A0103498401371B01400E
:102F4000114A63150906EFF07F9D93F9090863891B
:102F500009009387018798439306170094C318C408
:102F60008349C400E38A09CC371901401309094099
:102F7000C147232AF900114A914A232A590148409E
:102F8000FD19EFF07F9B232849014840EFF0DF9ABD
:102F9000E39509FE55B1232A9900EFF0FF99232804
:102FA000990048407D1AEFF03F995DBD232A4B41BF
:102FB00048407D19EFF05F9823284B414840EFF0DF
:102FC000BF9741B703498401B71B0140114A631EF3
:102FD0000904EFF0BF94930B000203AB0A00371C07
:102FE0000140914A1375FB0FEFF0FF91232A5C41DA
:102FF0004840FD1B5A99EFF03F9423285C4148401C
:10300000135B1B00EFF05F93E39E0BFC1375F90F4E
:10301000EFF07F8F232A5C414840EFF0FF91232897
:103020005C414840EFF05F910DB723AA4B41484007
:103030007D19EFF07F9023A84B414840EFF0DF8FE0
:1030400079B79387E4FFF59BD9EF83479401B9EBF8
:1030500003498401371B0140114A631A0906EFF046
:10306000FF8B83479401E38907BC93F92900E3951B
:1030700009BC3719014013090940C147232AF90047
:1030800093091002114A914A232A59014840FD1917
:10309000EFF09F8A232849014840EFF0FF89E3952C
:1030A00009FE59BE93F72900C5D7130A1002914AA9
:1030B000114B232A690148407D1AEFF0FF8723282E
:1030C00059014840EFF05F87E3150AFE51B7232A04
:1030D0004B4148407D19EFF03F8623284B41484043
:1030E000EFF09F859DBF83498401914A114B130ADC
:1030F000F0FD232A69014840FD19EFF0FF832328E2
:1031000059014840EFF05F83E39549FF09B1375714
:103110000020832747DA944363CC060294433706A2
:103120000080C205D18E94C3B78702402395A700C3
:10313000C1812394B70083C67700054593E68600D6
:10314000A383D700832747DADC472322F7DA82807C
:1031500001458280854789456316F5003715014092
:103160006F00607A371501406F00207A85478545EA
:103170006316F500371501406F00E0783715014000
:103180006F00A07837F7FF1F81471307D77E994656
:103190003306F740834506003306F5008507230014
:1031A000B600E397D7FE82803787002083270796F3
:1031B0003E952320A7968280411126C29547B78469
:1031C000024006C622C42382F40203D70402938776
:1031D00041877D8B39CF03C7070093168701E186AE
:1031E00063CB0600138451878346040091EA1307DA
:1031F00000F82380E700B2402244924441018280DB
:10320000137627006DF61367270093C646002380C8
:10321000E7002300D400B707008093870710DCD0B5
:103220002945ED2183470400C20793E7E711DCD06D
:10323000D9B703C70700930600086315D70023809A
:10324000070055BF83C651871384518799EA799B3C
:103250002380E70093C646002300D400B7840240D1
:103260005DBF1146E398C6FE759BDDB783C76187D6
:103270009DE3B7860020378700200326479A83A75F
:103280000696918F130630066377F60083A706969D
:103290002322F79A15B78280411106C6EF0030400D
:1032A000EF001026B2404101D1B7011185454145DB
:1032B00006CE02C202C402C61D278D472312F100AA
:1032C000C1473EC64C008D47371501403EC49D2B7B
:1032D000894537150140052D8545371501402525C0
:1032E000F24005618280B737002023AEA758B708A7
:1032F0000080814713030060130EF6FF63E3C700ED
:1033000082803388670213974700B306E50023A045
:1033100016012E9823A406012A8863F5C7014107E8
:103320003308E500850723A6060193F7F70FF9B7E1
:10333000B737002083A7C75903D78700B787024054
:103340002396E70003C7770013674700A383E700CE
:10335000374702408327078093E747002320F78001
:10336000828005455DAD011106CE2AC6DD3FB787D7
:103370000240A381070003C737001367B70DA3817D
:10338000E70003C7370013674700A381E7007D57B5
:103390002382E70003C757001367070CA382E700E7
:1033A00003C777001367070CA383E70003C7770001
:1033B0001377F703A383E700238C07003245034705
:1033C00055002384E70203474500A384E70203472F
:1033D00035002385E70203472500A385E70203475D
:1033E00015002386E70203470500A386E70203C70B
:1033F000970113671700A38CE70003C7A7017D8B14
:10340000238DE70003C7A70113670702238DE70099
:1034100003C7A70113670701238DE70003C7A701AF
:103420001377B70F238DE700F24013070060239F47
:10343000E700056182804111B787024022C426C29D
:1034400006C615472382E702054783D40702238275
:10345000E70203D40702C204C1804204418013770B
:10346000440029C3A1E02382070203D70702A16613
:1034700037440240558F420713670710D8D383277C
:1034800004801305401FED9B2320F4805D2C8327CF
:10349000048093E747002320F480B2402244924402
:1034A000410182802285EF00D0211374440213076A
:1034B0004002938761876314E402B786024003C722
:1034C000A60193F4040489C813671700238DE6004E
:1034D00011472380E700D1B71377E70FC5BF2380DB
:1034E0000700238A018655BF411106C622C4B7864C
:1034F000024003C446001374F40F93770404ADC76D
:10350000930700042382F600373500208327C5592E
:103510009843635B070403C756001377870755E793
:10352000D0471842635207049843E175FD1506071A
:10353000058398C398436D8F98C39843B70501C01E
:10354000FD151367073098C398436D8F98C303D751
:10355000E6008C43110742074D8F98C383578600BE
:10356000232EC5582396F6009377840091CFB75742
:10357000002003A747DA1C43860785831CC3B7874F
:10358000024021472382E7009377040181CBEFF0CB
:103590009FEAB787024041472382E70093772400E0
:1035A00091CFB757002003A747DA1C4386078583CE
:1035B0001CC3B787024009472382E700058811C46E
:1035C000B787024005472382E700B2402244410109
:1035D0008280411106C622C42A84EFF01FCD130554
:1035E000400685222285EFF01FD8378700209307F9
:1035F000079523280794378700201307879A378475
:103600000020B735002098C7B75600201305449610
:10361000DCC711469385055A23A2F6DAEFF0BFCC3A
:10362000B75700201304449623A087DAEFF05FD049
:10363000B2402244B7E700E03707002023A2E7109A
:10364000410182805D71930700603ECA9307405B31
:103650003ECC8567938747233ECE930720033ED019
:10366000930730023ED2B727550289073ED4B737B9
:1036700000009387C7163ED6B737000093874715DB
:103680003ED8B73700009387E7103EDAB7573412B9
:10369000CAC0938787672A894808A2C4A6C286C67B
:1036A0002EC632C4B68402DC3EDEEF00306D2A84C2
:1036B00019E92246B245A6864A85EF0010602A84A1
:1036C0002685EFF01FF12285B64026449644064930
:1036D000616182807325103482807325203482805A
:1036E00073253034828083A7418137177A0013070E
:1036F0000720B3D7E70293F7F70F238DF18613075F
:10370000803EB387E702239CF1868280B7F700E012
:10371000D8438146799BD8C303C7A1873306A70244
:1037200090CBD4CB98431367070198C39843136792
:10373000170298C3D843058B75DF9843799B98C3CC
:103740008280B7F700E0D8438146799BD8C303D77E
:1037500081873306A70290CBD4CB98431367070128
:1037600098C398431367170298C3D843058B75DF36
:103770009843799B98C38280797122D42A841165F9
:103780008545110506D6A12C930700202312F100D0
:10379000371501408D473EC44C00E14713050580B5
:1037A0003EC64D2022C837440140B70708000C0828
:1037B000130504803ECC02CA231E0100252E1305EA
:1037C000048085452921B25022544561828001112F
:1037D00026CAB744014022CC4AC84EC606CEAE899E
:1037E0003289014493840480634A2401F240624494
:1037F0004A85D2444249B24905618280930500045A
:103800002685CD2E65DDB387890083850700268553
:103810000504C205C181D12EC1BF138781811C431C
:10382000B78600209386464D3E95636BD500B7065C
:1038300001209386068063E5A60008C33E8582804A
:10384000FD57EDBF9C4513F7070113F8F70001C7BB
:10385000D8413368E80083D5050013F7F50F39C365
:1038600018418146854E3D4F930F8002930280049C
:10387000214E3396DE00B3F8C5006311160393980A
:10388000260033131F011343F3FF3377E300B3180C
:10389000180133E7E800639FF70550C98506E39AEE
:1038A000C6FD18C11307F00F6375B70454412146D4
:1038B000854E3D4F930F800293028004414EB39892
:1038C000CE0033F715016392E802131726000117A3
:1038D0003313EF001343F3FFB376D3003317E8003D
:1038E000D98E639DF701232A15010506E319C6FD4C
:1038F00054C18280E39457FA10C94DB7E39757FE3D
:1039000023281501DDB70CC982804CC98280371786
:1039100002405C439146B18B6389D706A146638B15
:10392000D706B7177A00938707201CC137160240C5
:103930005C4237070020130707009183BD8BBA97BD
:1039400083C607001C41B3D7D7005CC15442A18293
:103950009D8ABA9683C60600B3D6D70014C55442D2
:10396000AD829D8A369703470700B3D7E7005CC551
:1039700058423983937637001387C18136970347BE
:103980000700B3D7E7021CC98280B757E8019387C5
:10399000078061BF5C435843C166C983BD8B758F87
:1039A0008907C5466393D700C94701EF37470240EF
:1039B00003270780418B09CF37177A0013070720A9
:1039C00021A83717024058439316E700E3D606FEB6
:1039D00037173D0013070790B387E702B9B799C5BA
:1039E000371702401C4F5D8D08CF8280B717024009
:1039F000984F1345F5FF798D88CF828099C5371789
:103A000002405C4F5D8D48CF8280B7170240D84F8F
:103A10001345F5FF798DC8CF8280B7170240D84390
:103A2000B70600F0FD16758FD8C3D8437205598DBF
:103A3000C8C382808357050037370140130707C08A
:103A4000C207C1836304E502370700406300E50253
:103A500013070740630CE500371700409306078003
:103A60006306D500130707C06317E50003D72500D9
:103A700093F7F7F8D98F03D7650093F7F7CFC2070D
:103A8000C183D98F2310F50083D745002316F50293
:103A900083D705002314F502B7370140938707C089
:103AA0006316F50083C785002318F5028547231A9E
:103AB000F50082808357050091C593E71700231016
:103AC000F5008280C207C183F99BC207C183C5BFCD
:103AD0008357C50009C6DD8D2316B500828093C5C6
:103AE000F5FFFD8DD5BF93C5F5FFC205C181231834
:103AF000B500828083560501F577FD17F58F83D6D3
:103B00006500397122DC06DED58F03D7C500231886
:103B1000F5008356C500FD779387379FF58F83D6D1
:103B200045002A842EC6D58F83D68500D58F83D6AF
:103B3000A500D58F2316F50083574501C207C18321
:103B400093F7F7CFD98F231AF5006808EFF03FDC21
:103B5000B747014093870780B245631EF404A2571C
:103B60008356C4006547B387E702C206C186984101
:103B700063D5060406070356C4004206B3D7E7021E
:103B8000130740064186B3D6E702B3F7E702920671
:103B9000635706028E0793872703B3D7E70213F70D
:103BA0007700B367D700C207C1832314F400F25033
:103BB000625421618280925765B70A076DBF9207F0
:103BC00093872703B3D7E702BD8BD58FE9BF81C9A0
:103BD0008357C5000967D98F2316F50082800357E4
:103BE000C500F977FD17F98FC5BF93F5F51F2312AF
:103BF000B5008280035505006D8D3335A0008280AD
:103C000001A001A001A001A001A001A001A001A0AC
:103C100001A001A001A001A001A001A001A001A09C
:103C200001A001A001A001A001A001A001A001A08C
:103C300001A001A001A001A001A001A001A001A07C
:103C400001A001A001A001A001A001A001A001A06C
:103C500001A001A001A001A001A001A001A001A05C
:103C600001A001A001A001A001A001A001A001A04C
:103C700001A001A001A097D1FF1F9381A1BF17C18F
:103C8000002013012138178500001305E5FD97C5B5
:103C9000FF1F938525371386018663FAC5008322AB
:103CA000050023A0550011059105E3EAC5FE138523
:103CB000018697550020938525826377B5002320E0
:103CC00005001105E36DB5FEFD42739002BC8D4207
:103CD000739042809302800873A0023097C2FFFF66
:103CE0009382C23593E2320073905230EFC07FACC2
:103CF00097D2FFFF93828299739012347300203021
:103D0000EFC20FCB378400208327049641113EC6B3
:103D1000EF10C01A118963010512938741899843F6
:103D2000B246998E371700200327C7240583637690
:103D3000D700324798C3EF30B036EF30505A9384F3
:103D400001899840B247998F1307703E6376F70058
:103D5000EF200008B2479CC09387C1879843B246C2
:103D6000998E0567130777386376D700324798C373
:103D7000EF108047B717002093870721D84711CF4E
:103D80001387C1881043B246918E1306703E637646
:103D9000D600B246DC4314C38297B714002083A731
:103DA000841BB1C39387818894433247158F930650
:103DB000F07C63F9E600324798C39387841B9C4BE1
:103DC00091C38297938741889843B246998E3D6705
:103DD0001307F7A56379D70032479384841B98C3F0
:103DE000DC4891C38297324593840188B52C9C406E
:103DF00032471D8FBD679387F7A563F5E7000D2C4C
:103E0000B2479CC003C7118ABE841377F70F0DC752
:103E100003C7118A1377070C1DE3B717002083A788
:103E2000072999C3054582970327049623AEE188A5
:103E300093070004A380F18A41016FC0AFB903C7A3
:103E4000118A1377070415CB83A6C189032704962B
:103E50001389C189158F93064006E3FFE6FCB71767
:103E6000002083A7072999C30145829783270496D9
:103E70002320F900930700F875BF03C7118A620772
:103E80006187E35B07FA83A6C18903270496158F30
:103E900093064006E3F2E6FAA380018A71BFB757A2
:103EA000002083A707DA9C4363CC0700EFC24FB022
:103EB000371500201305052AEF1090106FC08FB141
:103EC0008280EFC2EFAEB717002093870723D85741
:103ED0003714002088D313674700D8D71189930778
:103EE00044279C4F1304442701CD99C30145829771
:103EF0005C4C99C3014582970545112A6FC08FAD6F
:103F000099C3054582975C4CF5DB05458297FDB763
:103F100037570020832707DA2320050091CB8146FD
:103F2000B705008090436357060099C22320F7DA53
:103F300001458280904313180601634608029043AE
:103F4000137606100DC290431376062009CE99C24F
:103F50002320F7DA98439C470A074983711718C151
:103F60005CC1054582808CC38546DC4765BFB75779
:103F7000002003A707DAB706008014C3584723A020
:103F8000E7DA8280EFC2CFA283C7118A93F7F70FD7
:103F900081E78547A380F18AB787002003A70796AA
:103FA0009387818909CB98C3B717002083A7472936
:103FB00082976FC02FA20547FDB7B717002083A7D0
:103FC00047290145A1C3B757002003A747DA1DCBF6
:103FD000144308479387818963D406028C43A16602
:103FE00089063788002093083006032608960D8E30
:103FF00063E4C800FD1681EA14438606858214C373
:1040000023A0070082801043E34106FED5BF378717
:10401000002003270796B71700209387C71A88A3A5
:10402000239107002392070098C7A380070082808E
:10403000EFC20F98B71400201384042A5C4041118A
:104040006C001385042A3EC623220400EF1020389A
:10405000B2476C001385042A5CC05C443EC6EF1076
:10406000003741016FC00F97B71700209387C71A19
:10407000982319E388C7828098479306703E3307D8
:10408000E54063F3E602EFC2AF92BA2388C79146D8
:1040900063F7E6000145EFF09FF76FC0AF930507A8
:1040A000BAA3EFF0FFF8D5BF8280EFC26F902A84E9
:1040B0000145EFF0DFF5B71700209387C71A11C845
:1040C000054798B3B7170020094723AEE7246FC010
:1040D0006F90A3800700E5BF828003288503630BF0
:1040E0000802EFC2EF8CFC5D014791C7050742074C
:1040F00041839C43DDBF83A7050891C7050742079D
:1041000041839C43DDBF81460146814502980145BC
:104110006FC04F8C0145828001458280EFC2CF86FF
:104120005C42032A85000329C5000049AA8488232C
:104130009C33B289A2075D8DEF10A079935565007D
:1041400093F5C503B305B0404E85EF20902E49E5A9
:10415000DC44984C03DB8900998F63F867014E8536
:10416000EF20103405456FC0AF854A9A4E8903563B
:10417000A900B30A8A40832B490063F4CA04568617
:10418000DE852285EF60E03B8357A9009844330425
:1041900044413E942286B3855B013A85EF60603AE4
:1041A0002A9403290900E31409FC4E85EF20502FBF
:1041B0009C4C80C8DA979CCC9C4093E747009CC0FD
:1041C00055B72285DE85EF60C0378357A9003E943E
:1041D000E39957FD8044F1B7014571B771CAEFB259
:1041E000BFFA832BC5001C4D035B8600BA8AB387D8
:1041F000FB40368A32892A8463F767013285EF20D3
:10420000302A6FB0FFFB1C450449B289BE9B03D620
:10421000A900338C9B4083AC49006377CC0662864F
:10422000E6852685EF60E03183D7A9001844B38482
:104230007441BE942686B3858C013A85EF60603068
:10424000AA9483A90900E39409FC4A85EF2050252C
:10425000032884036305080483451A0083470A0082
:104260001448A205DD8D83472A005A875686C20767
:10427000CD8F83453A002285E205DD8D02981C44EE
:10428000232C04001CC8B5BF2685E685EF60602B93
:1042900083D7A900BE94E39687FB04445DB7184C0E
:1042A0001C4004C85A9793E7470018CC1CC091BF24
:1042B00082801C49F9CBEFB23FED328AAE842A846A
:1042C0005DCE832A8500544503C76502835B860063
:1042D000B69A719BC20A2383E502328993DA0A01F6
:1042E0009399070193D90901338B3A410356A900E9
:1042F000420B135B0B01032C49006376CB065A86F5
:10430000E2853E85EF60E0230357A9001C44B30516
:104310006C0133075741BA99C20993D909013E8507
:104320004E86EF600022B307350103290900E31927
:1043300009FA184C1CC852855E9718CC18401367B0
:10434000470018C0EF20D015FE38184C2685B38BD7
:1043500077415C44239B7403998FDEB4EF20B078DF
:1043600001456FB0FFE53E85E285EF60801D035794
:10437000A900B307E500E31A67FB1C447DB70145BC
:10438000EDF22E85EF30803DE9BF7D558280EFB2A2
:104390009FE0B789002003C6018A138789458147BA
:1043A0009389894593F6F70F63E5C6006D556FB0A5
:1043B000DFE103280702938617001307C70363048E
:1043C0000800B687C5B71309C003338927032E84B5
:1043D0002A8A1306C0038145B38429012685EFB0DC
:1043E0003FE01305C9021146930544004E95EF6066
:1043F00040155E3080D8A685DCD083278A022285CE
:104400009CD4EF20907DB74500009385850D2285D3
:10441000EF20B07DB74500009385252B2285EF2046
:10442000107CB74500009385A50D2285EF20907B79
:10443000B74500002285054693858511EF20907BC6
:104440008D47DCCC95479CD09C20014593E78700A5
:104450009CC0B1BF19C93305A040B167938787B627
:104460001375F50F3E950821828001458280EFB2D9
:104470003FD49307C003B387F502378400201307A6
:1044800084452A89AE841306C003814513048445FC
:10449000BA973E85EFB0DFD4630709001306C00367
:1044A000CA85EF60000A9305C003B385B402A295E4
:1044B0009C459CC9DCC96FB0FFD1EFB2DFCD2A8A21
:1044C000371500204111AE89B2848145614613053C
:1044D000851B36C6EFB0DFD0B24637140020130973
:1044E0000423B68519461305C900EF6080051146FF
:1044F000D28513050423EF60C0041146CE85130551
:104500004900EF60000413040423A1E0B707000191
:10451000FD171CC4814483C7018A63CFF402EF10E6
:10452000003385475CD01567B71700209387472273
:10453000130707E298C31167130787A9D8C3254754
:1045400098C7014541016FB05FC81146A6851305A4
:104550008400EF50107F7DBF93F5F40F0145EFF01D
:104560001FF185044DBF1841B717002093874722DC
:1045700098C35841D8C3184598C782801855B75773
:104580003412938787676318F710EFB2DFC01C51AE
:104590002A8425456389070E371900201306400435
:1045A000814513050923EFB0BFC3B71400201306DC
:1045B000C002814513854427EFB09FC21306C00295
:1045C000A28513854427EF50D0779389442703A70A
:1045D00049014A869387442725EBB16603D786B401
:1045E000938686B4AE222E97CE22F6222E97369749
:1045F0009316270163DB0608D8CBD84B9356E70008
:10460000FD8A89EAB746F8FFFD16758FB7060500E3
:10461000558FD8CBD84B93563701FD8A89EAB746D8
:10462000F8FFFD16758FB7065000558FD8CBD84BC5
:104630009316670063CA0600B70600FEFD16758F65
:10464000B7060014558FD8CBD85311E73747000071
:10465000130707F1D8D3D44B014513D7E6007D8B60
:104660002380D18A9307062398CF13D736017D8BF9
:10467000130620033307C702D8CF1397660063548D
:1046800007000947B8C36FB05FB4F976FD16758FA0
:104690008966558F95B71305F00F8280514582804A
:1046A00003C6018AB7870020938687450147938711
:1046B00087456317E60081476313F702014582804F
:1046C00003A807036317A80009C50545EDD998A1FC
:1046D000828005071377F70F9387C703D9BFD05A96
:1046E0006319A60019C50545F9D993E707F89CA1F8
:1046F0008280850793F7F70F9386C60375BFEFB2E5
:104700009FA9378900202300050003C7018A4111B2
:104710009307894581441309894563179700130559
:10472000000241016FB07FAA9387C70383A647FEAB
:1047300063810618850493F4F40FC5B7B7170020FA
:1047400083A707236C003EC6EF20F00811469305AF
:10475000C4026800EF50F05E6C004E85EF209009B7
:104760001306C0033386C402B74500009385C51104
:104770004E854A96EF20F0099547371500206C00CA
:10478000232834031CD01305052AEF005044A685C6
:104790002285EFF0DFCD014569B709476390E70A4D
:1047A000EF50F009AA8963030512930AC402114667
:1047B000D6856800EF50F058324A370500F0EF1008
:1047C0006014337AAA00370500E0EF10A0136300ED
:1047D000AA04B71500209385052A6800EF10A05A97
:1047E0001DE5B717002083A7072312346C004E8500
:1047F0003EC6EF5080611DE1D68511466800EF503E
:10480000505452306C004E85EF50207B39A012344A
:104810009385C1844E85EF50405F01C5EFF09FC383
:1048200009B71306C0033386C402B7450000938559
:10483000C51D4E854A96EF5030003DBF0D4713050C
:104840001002E390E7EEEF30A0255C4412346C00D8
:104850005EB9B717002083A70723AA893EC6EF20B9
:10486000900D2A8A11C54E85EF20506F52857DB775
:104870009305C003B385B4024E85CA95EF20F03589
:10488000B74500004E859385850DEF20103695477E
:10489000A685228523283403232A34031CD0EFF075
:1048A0001FBD371500206C001305052AEF003032BC
:1048B000DDB504A1DC4DC4C12E84E39007EE0345B1
:1048C0008402EF20407EAA89E31A05E6454591BDA2
:1048D000EFB21F8E4EB52A84EF20F02001EDB7878E
:1048E000002003A7418A83A70796998F13074006E4
:1048F000637BF70083476402228593E72700230345
:10490000F402EF40504105456FB0DF8C83C7018A48
:104910006376F5041307C0033305E502B78700206B
:10492000938787453E95584D232C050050C50CC5EF
:104930000CC94CC98D476313F702085905C15A3990
:1049400093371600631CF700EFB29F86931506019C
:10495000C1814EB9EFF0DFF76FB0DF878280EFB231
:104960009F839307C003B307F502B7840020138722
:1049700084455D44BA97945315476398E60A1842F4
:10498000694445C72320060003AB8700D44783A9A9
:10499000870193848445C04B369B63733701BA8982
:1049A000B30A8B40328AAE872A8963F33A0999C5E4
:1049B0003E855686A285EF50D038AA8733855701A9
:1049C0009307C003B307F9024E9433046441A697DA
:1049D00083AA870009C52286D685EF509036569463
:1049E0009307C003B307F90223203A01A697984F13
:1049F000C0CBB309374123AC37016398090098470E
:104A0000D8CB98CB98436D9B98C31305C00333094B
:104A1000A9028D470144CA94D84C6318F7006396E5
:104A20000900CE248858EFF0BFEA22856FB0EFF975
:104A300091C54E86A2853E85EF50B0304E94E391ED
:104A40003AFB9307C003B307F902A697804749BF13
:104A5000B78700209387874581C91307C0033307B1
:104A6000E5023E97584B98C11307C0033305E50292
:104A7000AA97884F8280EFB22FF1004223200600D0
:104A800055C4AA876945D9C51305C003B387A702D2
:104A90003785002013058545B71A00208144AA9761
:104AA00003AB070393870A23BC43938A0A23898BAA
:104AB00099E39304700C9307805C63F487001304FC
:104AC000805C931C0401328A2E8993DC0C01130C48
:104AD000800C0146E6850145EF206021AA8929C99D
:104AE00048412286CA8523AE0A02EF509025CE8522
:104AF0005A85EF20405AAA8B4E85EF20601A83A773
:104B0000CA0399CB8504C204C180EFF04FB9E39288
:104B100084FD4D456FB0CFEA63D60B005E85EFF0A4
:104B20007F93CDBF23208A000145EDB76945DDB7EE
:104B30004545CDB7EFB24FE500422320060055C4EE
:104B4000AA876945D9C51305C003B387A70237856E
:104B5000002013058545B71A00208144AA9703ABAE
:104B6000070393870A23BC43938A0A23898B99E31B
:104B70009304700C9307005C63F487001304005CDB
:104B8000931C0401328A2E8993DC0C01130C800CD7
:104B90000146E6850145EF208015AA8929C94841CB
:104BA0002286CA8523AE0A02EF50B019CE855A85F7
:104BB000EF50803FAA8B4E85EF20800E83A7CA035B
:104BC00099CB8504C204C180EFF06FADE39284FD00
:104BD0004D456FB0EFDE63D60B005E85EFF09F872B
:104BE000CDBF23208A000145EDB76945DDB74545B6
:104BF000CDB7EFB26FD90329060023200600630664
:104C0000090EAA87AE8A6945A1C91305C003B387F7
:104C1000A7023785002013058545328B014AAA97E4
:104C2000845BB717002083A70727898B99E3130AB2
:104C3000700CB71900200144130C900C914C93890F
:104C400049277D5D050A420A135A0A0163188A0141
:104C500083270B00C9CB01456FB08FD69C48639862
:104C60009709EFF0CFA383D6640799E24545EDB7E6
:104C700083A70901858B99E3E3EA26FF03A749008F
:104C800063F3E6003687CA8B63732701BA8B1396EA
:104C90000B014182854691E38146D6852685EF400A
:104CA000C07D2A8426850DE4EF40F00683270B00A3
:104CB000330979412A84DE972320FB00DE9AE30C36
:104CC00009F883A70901858BB5FFEFF0AFF869B745
:104CD0006319A401EF40300483A70901858BBDF35C
:104CE00071B7EF4050032285CDB76945B5B75D4533
:104CF000A5B79307C003B307F50237870020130752
:104D00008745BA9703A8070215476307E800DD4700
:104D1000232006003E858280EFB28FC9D84F8D4791
:104D20006318F700EFF0FFECAA873E856FB08FCADB
:104D300001E7EFF05FD4CDBF89469307A00FE316DC
:104D4000D7FEEFF03FDFCDB7EFB28FC6A147AA8401
:104D50000021638AF50263ECB70085476381F502A1
:104D6000894713642400638EF5006FB0AFC6C14756
:104D7000638EF5009307000413640404EDB7136415
:104D8000140080C0DDB713648400E5BF4859136484
:104D9000040165D9EF20901CEDB7EFB26FC141114E
:104DA0009305F100AA84A3070100EFF07F8F15C5DA
:104DB000808793178401E18763D407021374F40793
:104DC0001307C0033304E402B787002093878745A5
:104DD0003E94232A04022320040241016FB08FBFB6
:104DE00083C7018AE37BF4FE1307C0033307E402A1
:104DF000B78600209387864513898645BA97D04F9A
:104E00000D47E31CE6FC84281306C00381453E855C
:104E1000EFB00FBDDD1493F4F40F0547636D9700F9
:104E2000C145EFF07FF29307C0033304F4024A94C4
:104E3000232804024DB718211367070418C1E5B7EA
:104E40003787002083C6018A130787458147638F10
:104E5000F6001307C703032647FC11CEB71700203F
:104E600093870723D85713670701D8D7B7170020B0
:104E700003C5C7258280850793F7F70FC9BFEFB237
:104E80002FB3EFF0FFFBB717002023AE07246FB05E
:104E90006FB483C7018A6371F5029307C0033305BA
:104EA000F502B787002093878745AA979843137523
:104EB000F70F118B98C3828001458280B7170020BD
:104EC00003C5072582809307C0033305F502B78722
:104ED0000020938787453E951C5995CF145115475F
:104EE0005D45639BE60285899A279DC1136787000C
:104EF0009AA73717002013074722144323A0D70A85
:104F00005443184723A2D70A23A4E70A0145828005
:104F10005D9B9AA7E5BF5D4582801307C0033307F9
:104F2000E502B7870020938687453697105395464C
:104F30006319D604EFB2CFA7045B585B938787450C
:104F4000630497005D479DE81304C00333048502A2
:104F500026853E94A28523280402EF20004893056D
:104F6000F00F2685EF20802E454709C9B745000080
:104F700048D89385E538EF20A04701473A856FB0C0
:104F80006FA55D473A858280B717002003A5872863
:104F9000358105898280B71700209387072305474D
:104FA0004111C8CB94DBD0DB8CDFD8D741018280A4
:104FB000B7170020054723A6E7268280EFB24F9F50
:104FC000B717002003A6072883A6018213178601BE
:104FD0006187630B051483C7818A614889483388D8
:104FE000070336980323C800631013150343150005
:104FF0008348050003280800220333631301834814
:105000002500C20833E3680083483500E208B3E8AE
:105010006800639B0811E207E1873E856FB08F9BB4
:10502000B3885702B69803AEC80063190607631722
:105030000E061398870113588841850793F7F70FD9
:10504000E3E0C7FE6317060193F81500FD57E386FA
:1050500008FC8989FD57F1F19377F80F636BC8005D
:105060009377F30F6367C300FD57E378C7FA93772D
:10507000F70F61473387E702BA9623A6060001CDF2
:10508000103118212206598E38214207598E3831A5
:105090006207518F98C2238806000DA863147E040E
:1050A0000DC9834E1500034E0500A20EB3EECE01CE
:1050B000034E2500420EB36EDE01034E3500620E34
:1050C000336EDE0183AE08006315DE012384F18AAE
:1050D00099B783C80801E3E2E8F71397870161876E
:1050E000468FA1BFE31B8EF415C5834E1500034EFA
:1050F0000500A20EB3EECE01034E2500420EB36EA4
:10510000DE01034E3500620E336EDE0183AE080011
:10511000E30EDEFB83C80801E3E1F8F31393870194
:1051200013538341C68F11BF3A883A83814F014F91
:105130008147E1428543094421B7EFB2CF859831D9
:105140009C2122075D8FBC21C2075D8FBC31E20725
:10515000D98F58416319F7000545EFE01FF5D9577E
:105160003E856FB08F86E5DF2E842A89AA85228549
:10517000B289368AEF0030417DF11C3004203705BA
:1051800000F0A207C58F2420C204C58F2430E2049A
:10519000DD8CEF002077E98C370500E0EF008076AA
:1051A000E38FA4FAD2852285EFF05FE1AA87E34975
:1051B00005FAE147B307F50203A501823E95894749
:1051C0005CC5232A25019387590013079500942372
:1051D0007D1714B39386F7FF6396F9002308050043
:1051E0008147BDBFB687E5B7B717002003A50728DD
:1051F00003A801820147E14809430546130EF00E5A
:105200006363A7008280B3061703C2969C2ACC462C
:10521000850793F7F70F9CAA63986500636AFE0001
:1052200005071377F70FE9BFE39CC5FEE37AF6FEA7
:1052300023A60600F5B71DC9CC41B83DBC2D2207F9
:105240005D8FDC2DC2075D8FDC3DE207D98F5841B1
:10525000B98F1845F98F99EBEFA29FF5138665007A
:105260008146E905EFF07FED6FA0DFF68280630FE6
:105270000514EFA25FF23A2693079002411132899A
:10528000AE89AA8463E8E7004A85EF1070214101E6
:105290006FA0BFF340420545034AF4007C24220A74
:1052A000336AFA000525E311AAFE034A34013C28BB
:1052B00013054060220A336AFA002925E316AAFC86
:1052C000034A14011C28856A220A13850A80336A5E
:1052D000FA00CD2BE31AAAFA034AD4005C24138502
:1052E0006A80220A336AFA00F12BE31FAAF8130A34
:1052F000C4011146D2856800EF50A024D4401306A3
:105300006401A5C6034774028347640222075D8FC8
:1053100083478402C2075D8F83479402E207D98FD7
:105320006395F60485466C002685EFF01FE1854AFB
:105330005C384828A2075D8D71238547630EF5020E
:105340008947E313F5F46C002685EF10E031B717B9
:10535000002003A7871B0DDB9387871BDC47E385B2
:1053600007F26C002685829705B781466C0026857A
:10537000EFF0BFDC814A6DBFE3880AF0094599234D
:1053800048A8218148B81146D28513056402EF5020
:10539000401B9385440011465285EF50801A9307B5
:1053A000540093855900F82BFD152380E70298A33C
:1053B0009831F8ABF8A31387F7FF6317F4009C4C00
:1053C000CA8526858297C9B5BA87F1BF8280EFA2C8
:1053D0009FDC2A89AE8901469305A0020D45EF1096
:1053E00010117D544DC94041AA840545E12948A8C2
:1053F000218148B89306E902930754001547938525
:1054000041841386C1837D5503C80600FD17FD1630
:10541000A38B07013388E50003480800A380070336
:105420003308E600034808007D17A380070103C87E
:105430001600A3830701E319A7FC11469305490051
:105440001305C401EF50E00FCE8511461305640229
:10545000EF50200F0545BD2168A48569218168B4FE
:1054600013850980852108A8218108B813054060AB
:10547000912928A8218128B813856980A121832733
:10548000890148A4218148B4A6854A8582972A8447
:105490002685EF10F00022856FA03FD3EFA2BFCF8B
:1054A0002E842A89AA852285B289EF00D00D01C5F4
:1054B00059556FA09FD11C300420370500F0A2077A
:1054C000C58F2420C204C58F2430E204DD8C1D2941
:1054D000E98C370500E03D21E38CA4FC18301C204A
:1054E00022075D8F3C20C2075D8F3C30E207D98FD9
:1054F000E1D385452285EFF07FACE34C05FAE14727
:10550000B304F50203A70182138A01828547269717
:10551000544799EA5CC7EFF0BFA9A2854A85EFF02E
:105520001FEBE38809F831A0E387F6FE7D55E3849D
:1055300009FE83270A000947A697D447E39BE6F6AE
:1055400003A44900138797001306E9029306540049
:105550008D070C237D17FD168CB20C227D16ECB244
:10556000E319F7FE056513050580A92E8327890138
:1055700048A4218148B4CE854A8582971DBFEFA2F9
:105580009FC1AE8441112A89B94526853284EF1026
:10559000406A631E0510CA852285EF00C07E631530
:1055A00005101C3083490400370500F0A207B3E75B
:1055B000370183492400C209B3E7F9008349340065
:1055C000E209B3E9F9003D2EB3F9A900370500E07F
:1055D000152E1020143038203C30639CA9081395F8
:1055E0008600518D4207598DE20785456C845D8D9B
:1055F0009305E0054C85392641811375F507C8856B
:1056000008301C2022055D8D3C20C207C98F283040
:1056100062055D8DC52C2181488608301C2022053D
:105620005D8D3C20C207C98F283062055D8DD92C65
:10563000C8863400C04095477D5613075400B38593
:10564000F6008C217D170CB3B305F90083C59502D4
:10565000FD176CB3E395C7FE0565130505809D2412
:105660008327890148A4218148B4A6854A85829769
:105670000DA8A206D18E4207558FE207D98F0327C6
:105680004900B98F03278900F98F99C78327C9007B
:10569000715581CB1304C9002686A2854A85EFF097
:1056A000FFDF41016FA07FB29386C18361B7795557
:1056B000CDBFEFA2FFAF5C412A84AE84C827DC37A0
:1056C000A2075D8D01249307058091CB85679387A1
:1056D00067806305F5022285EF10805C29A8A2850A
:1056E0002685EFF05FB5C9552285EF10805465F52A
:1056F000A6852285A52401456FA0DFAD228693856E
:1057000094022685EFF0BFB6FDB7EFA27FAAB717C8
:1057100000209387071D5CD193075006A309F5026B
:105720009307E006230AF502B75700009387E7576F
:105730005CC9B75700009387E7761CCDB7150020EA
:1057400099472A842304F502232E050019469385E0
:10575000952C13059502EF40D05E9307C05D1EB8EF
:10576000930730032309F40201456FA0BFA6EFA2FF
:105770003FA4B1642E8493841435EFF02FF4118983
:1057800015CDFD1485CCEFE05F832A897DD5AA87EE
:10579000814401E8CA852685EFE0CFFE01456FA070
:1057A0007FA332244C403E85EF40B0593A2400405C
:1057B000BA94C204B307E500C180E1BF5155C5B733
:1057C000EFA27F9DB717002083A78729AA89138599
:1057D000C18A9384C18A82978C40A5C983C7118AE4
:1057E0001384C18A93F7F70F81E78547A380F18A75
:1057F000C2050D46C1810D4503294400EF10204F1D
:105800002A8421C5AA84B224C840CA85EF407053B7
:10581000BE2484403E99E5F8EFE06FF55C40C82770
:10582000DC37A2075D8D79289307058091C78567CE
:10583000938767806318F50083A70901CE852285C9
:10584000829701C52285EF10A0456FA01F98EFA297
:105850003F9641113714002002C202C402C6EF0075
:10586000D0781305042AB715002019469385C5235F
:1058700013059502EF40F04CB717002003A707234C
:10588000938707231305042A3AC29847DC433AC496
:105890003EC623A6018C23A4018CEF10A0383758F4
:1058A0000000B7570000740030004C001308286B4C
:1058B0009387A77001471305042AEF1000314101B7
:1058C0006FA05F919317850021815D8D4205418115
:1058D00082809317850021815D8D42054181828000
:1058E0001357850193178501D98FB706FF0013174A
:1058F0008500758FD98F4167130707F02181798D56
:105900005D8D8280EFA2DF8AEFF09FFD6FA09F8CFC
:10591000EFA21F8A03A4C18CAA8401EC03A5818C89
:1059200011C5EF10803019C103A4818C22856FA0AE
:105930007F8A2285EF10602F05C198309C202207B6
:105940005D8FBC20C2075D8FBC30E207D98F584005
:10595000B98F1844F98FF9DB0040C1B7EFA2DF829D
:105960004041AA84AE891C300820A2075D8DEFF06B
:105970005FF631814205418191476306F500268536
:10598000EF10003231A41C300820A2075D8DEFF02B
:105990005FF419813C30137AC5032820A2075D8D7E
:1059A000EFF03FF3BE242A89E3EB47FD9E24E3E8B2
:1059B000A7FCD2852285EF40F03071F1CA8526859B
:1059C000EF10E046370500F0EFF0DFF3370500E0B9
:1059D000EFF05FF34E89054B930B04014A85EF10FE
:1059E000C02411E563130B12032909000DA29307CC
:1059F0004900EDDB83264900F5D618381C2822071C
:105A00005D8F3C28C2075D8F3C38E207D98F6382E7
:105A1000F604CA855E85852E0DED1C38834A040187
:105A2000370500F0A207B3E75701834A2401C20AF1
:105A3000B3E7FA00834A3401E20AB3EAFA00EFF06E
:105A40007FECB3FAAA00370500E0EFF0BFEBE39B71
:105A5000AAF858345C2422075D8F7C24C2075D8F2E
:105A60007C34E207D98FB9C3CE851305C400212E3B
:105A7000E31705F05C34034AC400370500F0A207C1
:105A8000B3E74701034AE400420AB367FA00034A56
:105A9000F400620A336AFA00EFF0DFE6337AAA0014
:105AA000370500E0EFF01FE6E30BAAECE30909EC91
:105AB00003497400682022093369A90011657D1526
:105AC000EFF05FE03375A90011C52685ED26AA84A5
:105AD00061C14041CE852685EF10604955E91C34EF
:105AE0000824A2075D8DEFF0DFDE1375F50F9947EF
:105AF0006303F50AC5476309F50885476312F50A8C
:105B0000CE852685EF40205D61A003A9C18C63147A
:105B1000390103290900014BE31209EC1C34082464
:105B2000A2075D8DEFF0FFDA1375F50FC547631E11
:105B3000F500B3074401A823BC33A2075D8DEFF045
:105B40005FD993074004630DF502854A1C3408248D
:105B5000A2075D8DEFF0FFD71375F50FC5476319E9
:105B6000F508229A83473A0003452A00A2075D8D73
:105B7000EFF03FD69307C076631CF5064E893DB71C
:105B8000E39809F2814AD9B7CE852685EF406004B3
:105B900001456FA0EFE2CE852685EF20B01DCDBF79
:105BA000CE8513050401C522E31B05DC1C3803491F
:105BB0000401370500F0A207B3E7270103492401D8
:105BC0004209B367F9000349340162093369F900F6
:105BD000EFF05FD33379A900370500E0EFF09FD2F3
:105BE000E30FA9D8C0C089452685EF40C07341BBEB
:105BF000E3910AE669B3EFA22FD9AA894289630F1C
:105C00000612AE8AD1453A8AB284B68B3E8BEF102B
:105C1000400279576311051203A44900A20B1C34FA
:105C20000824A2075D8DEFF0DFCA1375F50F336509
:105C30007501EFF03FC91357850018B408A4EFF0C1
:105C40005FC9218142054181220533656501420515
:105C50004181EFF03FC798309C2008A422075D8F58
:105C6000BC20218108B4C2075D8FBC3011651305CB
:105C70000550E207D98F13D787001CA818B813D78F
:105C80000701E1833CB838A83365AA00EFF09FC351
:105C900008A0218108B003D58900138A418BEFF059
:105CA0007FC228A0218128B003550A0023030400E5
:105CB000A3030400EFF01FC183570A0048A021810D
:105CC000850748B02310FA0063810A0203C71A004F
:105CD00083C70A0022075D8F83C72A00C2075D8F32
:105CE00083C73A00E207D98F99E713074900814734
:105CF00019C38327490013D787005CA458B413D76E
:105D00000701E18378A47CB423050400A305040003
:105D1000D1452285EF40007B28A4218128B48357F8
:105D2000090385C303D7890063FDE7002686CA857A
:105D30004E8585232A873A856FA08FC84441C104C8
:105D4000F9BF832749012686CE854A858297DDB72C
:105D5000EFA20FC601112A8432852ECE36CC3ACA64
:105D60003EC832C6EFF0DFBA09CDC2475247E2461D
:105D70003246F2452A882285EFF0FFE705616FA0E1
:105D80006FC57155E5BF18311C2122075D8F3C217D
:105D9000C2075D8F3C31E207D98F9386F7FF7557B5
:105DA0006366D70203C725030145098B0DC3D8419C
:105DB000630FF70094453D8F758F11EB13C5F6FF08
:105DC000E98F3385A7401335150082800545828011
:105DD000EFA28FBB03A4818BC544014B1389818B38
:105DE00019E06FA0EFBDFD1493F4F40FFDD87C3CD7
:105DF000032C040091C7FD177CBC228B6284CDB7B5
:105E000083294400814A03A549005C315821A20737
:105E1000D98F85EF18311C21514622075D8F3C2117
:105E200093058400C2075D8F3C31E207D98F5CC0C7
:105E3000EF40207185454E85EF4020504E85EF1094
:105E40008004AA8A4E85EF00B065832944006396DA
:105E50000902032709001C40631CE4042320F90005
:105E6000A2851545EF00B0461387618B1E235A8427
:105E7000B38A57412310570149B703A749004E85FC
:105E80001C33034A0700A207B3E74701034A270070
:105E9000420AB367FA00034A3700620A336AFA001B
:105EA000EF00707EAA9A4E85EF00905FD28945B7C9
:105EB0002320FB0075B7EFA22FAD44412A899C3007
:105EC0008820A2075D8DEFF0DFA019811375C5034F
:105ED000D1476312F526FC30E820A2075D8DEFF074
:105EE0005F9FBC302A8BA820A2075D8DEFF07F9EBC
:105EF0009C30AA8C8820A2075D8DEFF09F9D2A8C94
:105F00004A85EF005078B717002083A7472803D7AA
:105F1000618B2A8D8D832A97FD8B9389618B63EC2E
:105F2000E72003A4818B814A138A818B1DE81545E4
:105F3000EF00F0372A846300052071468145130580
:105F40004400EFA0EFA98D477CBC83270A002320E3
:105F50008A001CC05146A68513058400EF40605E90
:105F600095ACD834DC2422075D8FFC24C2075D8FFA
:105F7000FC34E207D98F58486316F70298389C28FA
:105F800022075D8FBC28C2075D8FBC38E207D98F1E
:105F9000184C6319F700DC30D4205A24A207D58F9F
:105FA0006306F720A28A004051B7CC4203C85500CF
:105FB00003C34500220833686800637C060D93D54F
:105FC000860094A38CB393D50601E182ACA3B4B34D
:105FD000630E072A74336C23A206CD8E6364D61435
:105FE0006362A814935689002300270114B39356C3
:105FF00009011359890134A3A3012701782C014B0E
:10600000058B630F0718638D081858404443D83038
:10601000D4202207558F6315071894339823A206BE
:10602000D98EB8234207D98EB8336207558F61E7FE
:106030005E2C03C904005146D1075EAC9C30930529
:1060400084002685A207B3E7270103C9240042097B
:10605000B367F90003C9340062093369F900EF40FE
:10606000404E4A2CEFF01F86A8A02181A8B02383C0
:106070000400A383040023850400A3850400D14504
:106080002685EF402044A8A42181A8B4032B440016
:10609000D5A063090609F43103C36500A206B3E67F
:1060A00066006361D60801CB742378332207558FCD
:1060B0006303E8008148983194212207558FB42169
:1060C000C206558FB431E206D98E2E8765AA935643
:1060D00089002300270114B393560901135989013C
:1060E00034A3A3012701742378332207558FE307D4
:1060F000E6F0814821B75443EC23F833DC32D02258
:106100002207A2074D8FD18F631AF7029C32982283
:10611000A207D98FB8224207D98FB83262075D8FA4
:10612000B68731B74A85EF00105683D7090033850B
:10613000A7402390A9004A85EF009036014B8DA01F
:10614000B1554A8583244900EF00B02ECA855A858F
:10615000EF0030559C3003C90400A207B3E72701C4
:1061600003C924004209B367F90003C93400620976
:106170003369F900E31609FC03270A001C40631485
:10618000E4022320FA00A2851545EF0050145A8539
:10619000EF00704F83D709003385A7402390A900F3
:1061A0005A856FA0EF8123A0FA00F1BFFC30E820F0
:1061B000896BA2075D8DEFF0CFF1FD1B3375750183
:1061C0004205418101E96A24EFF0AFF033757501B2
:1061D000E31205D883D709003E9D2390A901FC3026
:1061E000E820A2075D8DEFF0CFEE9317250163C283
:1061F000070213153B017C2C4D810E05135C6C00CE
:106200006695137CCC0393E71700330585417CAC7E
:106210004AAC83244900BC30A820A2075D8DEFF072
:106220004FEB9C302A8B8820A2075D8DEFF06FEA40
:10623000FC30AA8BE820A20793DB6B005D8DEFF0AA
:106240004FE94E054D81131635003305CB0013FB86
:10625000CB03832749003305654142051357860068
:1062600041815440D8B313578500F8B32380070009
:10627000A380070023810700A3810700D0A3E8A320
:1062800085480147E39306D2E31307E42322240160
:10629000B5B3EF92FFEE032C4500011132CA03475C
:1062A0007C00AA8D03456C00220783DB0503598D12
:1062B000AE8CEFF00FE28966B377D500138ACBFE80
:1062C000A146334ADA0283D48D0009677D173EC6A2
:1062D0003379E500B1144209C20413590901C180A0
:1062E0000144514D3ACC420A135A0A0193163A001E
:1062F00093970601C1833EC89387DBFE3ECE89E4B7
:10630000014505616F909FEBE247A68A337BF90058
:10631000B24733EB6701F24763C6F400C24A8967AC
:10632000336BFB000146D1450945EF00501CAA899B
:1063300039C948415146E285EF40A02003A64D00EF
:1063400083AB49006A9623A2CD0003D6AD00B30605
:10635000A6412395DD00568D63090D0403D4AD00DD
:1063600063738D006A844204418001E483AD0D00B3
:10637000E5B7814509460D45EF007017AA8511E57F
:106380004E85EF00F0117D55ADBF03A64D0002A56F
:1063900022A550C14E85EF00D030B3068D40139D2D
:1063A0000601135D0D01E3130DFC5A85EFF08FD14B
:1063B0002383AB002181A383AB0013854A014205EF
:1063C0004181EFF02FD02381AB002181A381AB006D
:1063D000D14523850B00A3850B005E85EF40800E21
:1063E00003A74C0152462385AB002181A385AB0056
:1063F000CE8566850297B384544152994E85C20476
:106400004209EF00F009C18013590901228DC5BD71
:106410003C296385B7002CA9A309050082805E2D65
:10642000184DB306F7002388B60E9386270085071C
:10643000C207C18356ADBA972388C70E82805A2DF2
:106440001C4D9306170056ADBA972388B70E82806D
:106450005E2D184D13D68501B306F7002388C60EAE
:1064600093861700C206C182BA9613D60501238807
:10647000C60E93862700C206C182BA9613D685003F
:106480002388C60E938647008D07C207C18356AD89
:10649000BA972388B70E828015C15E2D184D13065A
:1064A00030049386170056ADBA97FD562388D70E51
:1064B0005E2D6376F60093F6370091E28280938634
:1064C000170056ADBA972388070EDDB7630C051683
:1064D000EF921FCE03290502DD5763020916AA8435
:1064E0000146930540130145EF007000232AA900DF
:1064F0002A87FD5763050514834639019387418236
:1065000081E69443850694C3404388438547232C02
:1065100089002320A9001CA01CB099473CA0A3011E
:106520000400EFF0EFBB9357850048A05CB0935791
:10653000050161817CA068B00324890129472304F7
:106540000400A304040023050400A305040023069B
:106550000400A306040023070400A30704008347E4
:1065600029016388E700F11793F7F70F0547636A7E
:10657000F700DC205CA4DC305CB4FC207CA4FC30A4
:106580007CB423080400A308040023090400A30921
:106590000400230A0400A30A0400230B0400A30B35
:1065A0000400230C0400A30C0400230D0400A30D1D
:1065B000040083C584028147414613970701418344
:1065C00081466376B7003387F4008346970233072A
:1065D000F40054AF8507E392C7FE1307C402930784
:1065E000C406230007000507E39DE7FE1307C40E5A
:1065F000238007008507E39DE7FE37558263130577
:106600003536EFF0EFAD935785002306A40EA306B1
:10661000F40E032689019357050161812307F40EC7
:10662000A307A40E231E0900814713074004B306E5
:10663000F6002388F60E8507E39BE7FE81473E853B
:106640006F905FB9D9573E85828011CDEF925FB6CA
:10665000005101C8484811C1A125232A0400232C58
:1066600004006F903FB7828063000518EF925FB41B
:106670000051630904163828A1476315F7169831AD
:106680009C2122075D8FBC21C2075D8FBC31E207D0
:10669000D98F18546398E714AA84B1452285EFF086
:1066A0003FD72685EFF09FE2631905120546930553
:1066B00050032285EFF0BFD691452285EFF03FD8F9
:1066C0001146930520032285EFF07FD50854EFF0A3
:1066D0006FA3AA852285EFF0BFD71146930560030B
:1066E0002285EFF0DFD34850EFF0CFA1AA852285B5
:1066F000EFF01FD61D469305D0032285EFF03FD261
:106700005E2C184C05462285B306F7002388C60E7A
:10671000138627004206418252AC9386170083C538
:106720009402C206C182BA962388B60E93863700B9
:10673000C206C18256AC83C5A4023A96BA96230813
:10674000B60E138647004206418252AC83C5B4029E
:106750003A962388B60E93865700C206C18256AC7D
:1067600083C5C402BA962308B60E13866700420694
:10677000418252AC83C5D4029D0732972388B60E5E
:106780005EAC83C7E4022308F70EEFF0FFD04E2C77
:1067900048489385050FC205C181512D03478402E6
:1067A0001C4C4C484840D8A70347940203A9440016
:1067B000D8B70347A4029306300413860185F8A7CF
:1067C0000347B402F8B723A204002687EF30806D98
:1067D000268523A22401EFF05FE73C3885073CB80B
:1067E00085477EAC6F901F9F8280EF927F9C11281F
:1067F000BD24B717002083A7872191C382976F908C
:106800007F9D375700201307B7DA719B23A0E18CD7
:10681000B717002083A7C727231107008D07F19B17
:1068200093960701C182BA9716A32302070023A2F9
:10683000F18C0546D0A396A3B6A323AEE18A82804D
:1068400049C183A7018C636EF50683A5418C637AE9
:10685000B50683A6C18B130685FF230E05FE13879D
:10686000C18B6373D60010C3835685FFBE96630445
:10687000D60203C8460063100802638ED5000C439D
:106880006393B60010C38E22231CB5FE9622B30577
:10689000F640BE96AEA28355A5FFB386B70063024D
:1068A000D60203C84600631E0800032807006313CE
:1068B000060114C3035785FF9AA2035785FFBA97B1
:1068C000AEA382808D05C205C181F199C205C18147
:1068D0003147AE8763F3E500B14737170020032641
:1068E000C727C207C1830D06719A6360F60A03A722
:1068F000018C636DE50883A6418C6379D508930606
:1069000085FF835885FF998EC206C182938588FFD3
:10691000958DC205C18163EAF5066389F5063303E7
:106920001701034843006314080293858600138807
:10693000C18BAE97032E0800C207C18383580300A2
:10694000B305F70063166E022320B80015A0138864
:10695000470163ED050393858600AE971388C18BCD
:10696000C20703230800C183B305F700E3EE65FC0B
:1069700023901501B6A123820500231CF5FE962164
:106980006306D60036973EA382800145828039C5D2
:106990001307350042074183719B42074183B1468B
:1069A000BA876373D700B147371700200326C7277C
:1069B000C207C1830D06719A01456362F60203A7FF
:1069C000C18B83AE018C9385C18B3303F640B30634
:1069D000D741C206C182615E63E4660001458280E0
:1069E0003385DE0003484500835805006317080619
:1069F0003308DE4046986362F806138347016362FA
:106A00006804A107B697C207C1833388FE0023102C
:106A100018012311D8002302080085461EA154A1A5
:106A2000835608006304D600F696BEA26319A70039
:106A300083A6418C8147502301EE91C398C1210563
:106A4000828085475CA1DDB71A2385477697E5B735
:106A5000E39CE6FEEDD794C1DDB7C686B5BF83A53E
:106A6000818283A6C182B76700209387F7FE37171C
:106A70000020F19B1307872D1385060103D805001D
:106A80002320070001466318C800890611078905FD
:106A9000E396A6FE8280832807000506420623A00F
:106AA000170183D806001CC34182C697E9BF9D47E2
:106AB00063EDA700B71700200A059387872DAA97D3
:106AC000884309C5184198C382800145828099C9CD
:106AD00093172500371500201305852D3E951C4181
:106AE0009CC10CC18280EF920FEB98319C21AA844B
:106AF00022075D8FBC212E84C2075D8FBC31E20767
:106B0000D98F5841639FE70018301C2022075D8F02
:106B10003C20C2075D8F3C30E207D98FDCC06F900C
:106B2000CFEA03A5818D01499309400605C11841AB
:106B3000DC40032AC5006311F7048545EF00705857
:106B40009307190093F7F70F63F7290383A7018EC3
:106B5000C5DF984319CFD440631DD70014301820E7
:106B6000A206D98E38204207D98E38306207558F59
:106B700098C3DC47F1BF3E8952854DBFEF924FE38A
:106B8000411132C636C42A84EFF0FFF53246A246E0
:106B9000814719CA18321C2222075D8F3C22C20786
:106BA0005D8F3C32E207D98F1CC4814799CA983265
:106BB0009C2222075D8FBC22C2075D8FBC32E20798
:106BC000D98F5CC441016F90EFE0EF926FDE58CD3A
:106BD0001387018D834807004111232205002324D8
:106BE000050023260500230905022320050213833F
:106BF0001800A30A1503232805012A843EC6230092
:106C00006700EFF0BFF7B2472285829711E99387BB
:106C1000C18C984318C080C3228541016F908FDBDF
:106C20000144DDBF23A4A18C82800345250305898F
:106C30008280AA870145A5C5BDC31396050141827F
:106C4000328863DB05003308C040BA274208135876
:106C50000801054563650705D427D84381C60D455E
:106C60006391A6020D8F9386070105456369D702DC
:106C7000D8C3BA2701453297BAA79A273A9692A75E
:106C80008280FD16C206C1828548054563E9D800A9
:106C900063D70500B62763E406010D8FD1BF82805C
:106CA000EF926FCF01440DCDAA8501440D4985496E
:106CB000FE25FD17C207C183FEA59DE3DC258441A7
:106CC0001D4563882701FD17C207C18363EDF900E5
:106CD0001945EFF0DFDF05041374F40FA685E9F81A
:106CE00022856F908FCE2E85EFF09FB5EDB7EF9296
:106CF0008FCA8547630DF50031C589476306F504E2
:106D00008D476305F504014422856F900FCC8144C3
:106D1000D104B904C204C1808947B2892E8963E9CC
:106D2000C70279CA1945EFF09FD82A8469DD23226A
:106D30000500231425012315250123200500230622
:106D40003501B5A0D144E9B78144E1B78144E9B741
:106D50008D470144E31AF6FA1D45EFF05FD52A840A
:106D60005DD1B3079500CD07F19B371700205CC1BB
:106D700093074727DC438D04F19893879703F19B92
:106D8000230635012320050023142501B3849740F1
:106D90009309472763739900CA84854726A47EA474
:106DA000B30499400D4A2289854A6347900085477C
:106DB0007EA4A306040089BF1D45EFF05FCF09E55F
:106DC0002285EFF0FFED81B783A749002316450127
:106DD000232005002320A9009387970306A5F19B94
:106DE00063F3F400A687130705013EA558C12317D6
:106DF00055019D8C2A8955BF938735001385340131
:106E0000F19B71993E9542054181EFF05FB82A846C
:106E1000E30B05EEAA94CD04F19844C12314250197
:106E200023152501232005002306050049B71E254B
:106E300063FAF504EF92CFB72A84AE84B387F540A6
:106E40002E2463E995025C2481EF638B95004C400E
:106E50002285818DA695C205C181EFF0BFA62A8447
:106E6000084026A406A419C1EFF09FE323200400E4
:106E70006F904FB61A248D8CC2043E971AA4C1801D
:106E800000407DBF8280814719E13E858280850771
:106E900093F7F70F0841CDBF01C57E2585077EA575
:106EA000828009CD99E182803A859E251625184178
:106EB000B697C207C1831EA565FB0CC18280EF9205
:106EC0002FAF2E84EFF0FFFD2285EFF0FFFC6F90D7
:106ED0006FB03DCDEF922FAC2A84AE845955ADC52D
:106EE0001A249E256362F7060149014A8359A400CA
:106EF000BE24B3894941B387274163C9F9049399F3
:106F000007014840CC4093D909015295CA954E8655
:106F1000EF3020634E9A3E24420A4E994209135A9A
:106F20000A0113590901639447010040014ABE2434
:106F30006365F900844099CC0149BA249E24631604
:106F4000F7029C409DC35D556F902FA8C20955BFA5
:106F50005955828009C801493A241E246314F70058
:106F60001C40F5F3C1F40145C5B77DF441B7EF927C
:106F70008FA203294500AA89834799000345890008
:106F8000014AA2075D8DEFE0DF94937AF50F03A429
:106F9000418D31099384418D01E401456F90EFA249
:106FA0001C280145639457035C488DC3084CCA866E
:106FB0004E86A285829719C963080A005C4423267D
:106FC000FA009C4080C05CC4054581495C44228A2B
:106FD00071F53E84D1B7814799C998319C21220728
:106FE0005D8FBC21C2075D8FBC31E207D98F1CC108
:106FF00001458280814799C998319C2122075D8F84
:10700000BC21C2075D8FBC31E207D98F5CC101454D
:1070100082804CC910CD8280EF92EF97AE842A898E
:10702000D1452685B289EFF0DFC015C901468145FB
:107030000545EFF0DFCB2A8409E57D594A856F903D
:10704000CF98A685EFF0BFE74E85EFE07F8C19ED76
:107050007159E30594FE2285EFF09FC4C5B7B15581
:107060002685EFF01FBD71F92684F9BFCA85630537
:1070700009008327090099E3930545008347090127
:107080000347A9008346B9002A884E862285EFE08F
:107090009FB62A897DBFEF92AF9113064500EFF0AE
:1070A000BFF76F902F93EF92AF90AA840145EFF056
:1070B0001FA02A8411CD71468145EF906F929307EE
:1070C00000F83CB49387418D984304A880C358C40A
:1070D00022856F902F906D55828083A6818D03A6A7
:1070E000018F83A5018E03D54183938741831307C5
:1070F0001500131507011318070141816353080098
:107100000565368719E7328719EB2E8719EF8AA3B1
:1071100082800358C701E30CA8FC5847E5B7035821
:10712000C701E306A8FC5847C5B70358C701E300E9
:10713000A8FC5847E1BF1C4963960710EF92AF8542
:107140004111AA84328411E62EC6EFF01FF9B24530
:107150002A8403A7018E31E703A7818D25EB83A93C
:10716000C18D1389C18D4E8759E783A7018FCDEB60
:1071700085C198319C2122075D8FBC21C2075D8F9C
:10718000BC31E207D98F89C711462685EF30603BB5
:10719000C2AC23A6340123209900014541016F9020
:1071A000CF825E2F63928702104359CED1CD9431A6
:1071B0009C21A206DD8EBC21C207DD8EBC31E20718
:1071C000D58FD9C36302F608584771B75E2F639213
:1071D0008702104335CAADC994319C21A206DD8EC9
:1071E000BC21C207DD8EBC31E207D58FB1CF630D64
:1071F000F6045847A5B75E2F63928702104329C64D
:10720000A1C594319C21A206DD8EBC21C207DD8E72
:10721000BC31E207D58F8DCB6308F6025847A9B77A
:10722000DA2F631F870094319821A206D98EB821E6
:107230004207D98EB8316207558F94436386E600C2
:10724000DC4735B74D558280555589BFEF825FF6D3
:107250001C49411191C70144228541016F809FF76C
:107260002AC60D45EFF0BF842A8475D5B245138731
:10727000C18D9C4D1CCDDE2D5EAD85471CC99E2564
:1072800093E727001EA5BC353CB5BC253CA59C4119
:107290001CC11C436394B702DC451CC323A6050034
:1072A0000945EFF0DF82B77700009387670D1CD0A8
:1072B0009387018E984380C358C479BF23A6F18E6B
:1072C00081461387C18E89E7F1DA23200700F9B7D9
:1072D000D0476317B60091C21CC3D845D8C77DBF3D
:1072E0008546B287CDB7AA870358C5021459D23B49
:1072F0000C5583D807043305D84005822E95328774
:1073000063F3C8004687420741833307E54063457E
:1073100007002397070382803387D5406356E00038
:1073200023970702014582808D8EF6B7E5BFEF8275
:107330003FE85E352A84BE95C2055E39C1814EB5EF
:1073400063F3B7005EB52285EFF0FFF95E388983FD
:10735000634BF50083476402228593E727002303EC
:10736000F402EF20401B6F80FFE6EF827FE44111C3
:10737000014409CDAA854841014411C52EC6EFF04C
:107380003F92B2452A841145EFF06FF42285410106
:107390006F805FE4EF82DFE1014401E522856F80C9
:1073A0007FE30441EFF07FFC2A941374F40F2685E9
:1073B000EDB7EF82FFDF41112AC61145EFF02FEF45
:1073C0002A8401C9B2455146EF30A0174840EFF07A
:1073D000BFAC228541016F80FFDF0CCD8280232866
:1073E000B50882802326B5088280232EB5088280C6
:1073F0000CD18280232CB508A30EC50282801C49C3
:1074000005476374F70429476381E704EF825FDA75
:107410002A840325850809C5EFF09F8823240408E2
:1074200003254408FD577EBCEFF0DFF6685C23229D
:107430000408EFF03FF603250408EFF0BFF5232E14
:107440000406232004086F80FFD88280EF825FD378
:1074500037190020930709231387418E83CC8701B6
:107460001C43316B850703A4818D1CC393096006FF
:10747000814A130909239384418E138A818D094D12
:10748000130B8BB9938B418509E803A4018F938477
:10749000018F631C04226F807FD2FD1993F9F90FCD
:1074A000E38B09FE034624051448854D6382CC0214
:1074B000834D040B63800D100327C40AB386BB0100
:1074C00083C6F6FF05072326E40A6378D70C814DAF
:1074D00018489946631DD700105C9440918E03268E
:1074E00089016376D60093871D0093FDF70F16245C
:1074F000014CA18A95CE91466305D7009D4663193C
:10750000D7020328440A8326840A0325040A832514
:10751000C901B306D8029040185C198EAA96B3D65A
:10752000B60263F9C61093871D0093FDF70F054C53
:107530000325440819CD185C94401946998E031709
:1075400004053307C70263E6E600EFF0BFE4232239
:10755000040818488D466312D710145C9840158FA4
:107560008326890163E6E61063940D108347C40304
:107570000347D403850793F7F70F230EF40263EB59
:10758000E70083278409230E0402639A07122285E9
:10759000EF107078A28A4044C5BD2326040A19471B
:1075A0006366B70193871D002308F40A2285EF2044
:1075B000205531BF0317E4036344070005077ABC75
:1075C00003270408E30507F08315E4030317040504
:1075D000E35FB7EE6384A6030317C4048316E404D1
:1075E000B1470D8736979376F60F63F3C700B14620
:1075F000DA9694223317D7002318E4048356A4059F
:1076000003574406231F040263F3E600368742074C
:107610004183835604040583231EE4046376D70064
:1076200013971600231EE404231DD4042285EF20A3
:10763000003679BD0347140B014C330707032A9723
:107640003357B702E376C7EE2285EF208045034724
:10765000140B0507A308E40AE1BDA546E316D7F01D
:10766000185C9440998E032789010607E37ED7EEC4
:107670002285EFD08FF22285EFF07FD85C44638DB6
:107680000A0223A6FA008327C40981C7084CED55D6
:107690008297630B0C005E305A2C0C5428509306D2
:1076A00044002286EF20201E032CC400A285094539
:1076B000EFF0EFC16284C9BB2320FA00E9B7084CA0
:1076C000A2858297E30505ECF1B52285EFD0EFECBA
:1076D0002285EFF0DFD20329C400A285094523A04B
:1076E00024014A84EFF0AFBE6DB3EF827FAC1C4142
:1076F0002E846390B704DC451CC123260400228538
:10770000EFF0FFCF1C4829476381E7020547638EEE
:10771000E7008347640213F7170001CB93E72700C4
:107720002303F4022285EF10105F232804006F80EA
:107730007FAA23A6F18E81461387C18E89E7D5DE05
:10774000232007005DBFD0476317860091C21CC38A
:107750005844D8C75DB78546B287CDB71C491D4789
:107760006365F70AEF82DFA431678A07130787B7DB
:10777000BA979C432A848287EFD02FE21387C18D6A
:107780001C43639987005C441CC323260400A28524
:1077900009453DA823A6F18E81461387C18E89E74E
:1077A000EDD623200700D5B7D0476317860091C2D6
:1077B0001CC35844D8C7D1BF8546B287CDB7EFD0D8
:1077C000CFDDA2851385018EEFF03FF2A2850D4536
:1077D000EFF0EFAF014531A8EFD02FDCA285138584
:1077E000818DEFF09FF065B78545EF10B047954765
:1077F00001C96F803F9E8545EF10D0467DF9A547B2
:107800001CC82285EF103051F1B701458280EF820C
:107810003F9A41112E8511CE0E2632C6EFF03FB1B0
:1078200032463285EFF0CFC781473E8541016F80F8
:107830007F9A8147FDFAEFF07FF2AA87FDB7EF82CA
:107840003F9703A4818D9304500619E06F809F98A1
:107850000326840819CA832704098146A2858DCF8F
:10786000084C829719E123240408FD1493F4F40FC3
:10787000F1DC8347640213F7170009CF93E7270071
:107880002303F4022285EF10104983476402F19B21
:107890002303F402404455BF0145EFF05FF7D9B729
:1078A000EF821F91EFF0BFF91387818E1C238507AC
:1078B00093F7F70F1CA3858B99C3EFF03FB96F8047
:1078C0007F91EF827F8C1849A94741112A84631E5A
:1078D000F700AA851385018FEFF03FE1A2850945E6
:1078E000EFF0EF9E41016F80BF8D1C412E8B03296D
:1078F00005063EC65C4183298502035AC5013EC484
:10790000835A45028324C509832B8501EFD0EFC834
:107910001385818DA285EFF05FDD0325040819C171
:10792000EFF05FA7685C19C1EFF0DFA603254408FC
:1079300019C1EFF03FA6A2850945EFF04F9981C428
:10794000ED555E858294E30F0BF8D687528734009D
:107950007000CE854A85EF10107369B79387018355
:10796000884303A7418E3A9588C38280EF82BF8205
:107970002A890945EFF0AF93B71400209384442778
:107980002A8425E19C488983858B89E701442285E7
:107990006F80BF8383A7018F03A6418E0145814677
:1079A0009389418EF1E701C58545EFF09FF10945C7
:1079B000EFF0EF8F2A8415E583A7818D03A50900D9
:1079C0007D191379F90F1306F0078145DDEB09C422
:1079D00085452285EFF0FFEE0945EFF04F8D2A84B3
:1079E00055D51306400B81452285EF806FFF930725
:1079F00000045CA89C44231C040613078021231B5D
:107A0000F4065E385EB47EB4E1773EA4DC40637475
:107A1000F700930780212310F404C1677D577CC4CD
:107A200085472318F4047ABC231DF404EFF01FF3F8
:107A300083A7418E68D428D01CDCB78700009387C9
:107A4000E7802328F408B717002003A7472293876D
:107A5000472268C82320E40AD8439C4728D8230E2D
:107A600004022322E40A2324F40AA308040A05B723
:107A7000985F3307E6406364D700BA863E85DC47EB
:107A800015B7D42B636CD900636AD600985F3307AF
:107A9000E5406365B7003686BA853E84DC473DB76E
:107AA000EF820FF113050004EFF05FEC6F808FF2AF
:107AB000EF820FF02A842E85EFD09FE511CD1E397D
:107AC00081CF938787FD3E87C207C1836373F4002C
:107AD000228713140701418022856F80AFEFEF8268
:107AE0002FED03A4018F9384018F19E06F808FEE37
:107AF0002285EFD08FAA2285EFF07F900329C40062
:107B0000A285094523A024014A84EFE05FFCF1BF70
:107B1000EF826FE81C49AA842E8AC827DC37A207A7
:107B20005D8DEFD01FDB058929E94169130909FC47
:107B300003270A0103A68190DE2454334C23B29715
:107B4000A206D58D7423C206CD8E6C33E205D58D89
:107B50008356CA00AE96B386D74063D506028D8F92
:107B60006359F000918DC205C840C181CEA4EFF0E9
:107B70000FAC23A044016F804FE55285EFF09F8149
:107B8000014AC5BF5C374827A2075D8DEFD07FD47F
:107B9000058915CD9C48C037C8272204498C4A85E1
:107BA000EFD05FD29C48698CC827DC37A2075D8D77
:107BB000EFD03FD21375E50313651500EFD09FD0CA
:107BC0009C48418D42054181C8A72181C8B7032443
:107BD0000A005285EFF06FF945D4228A91BFEF82F7
:107BE000AFDA83C7818F2A84C18B13898190F1C753
:107BF0008325090038558356450670553305B7402F
:107C000083A7418F9384418F634405026316B700B5
:107C10003307F640634E0700631EF60203A5019189
:107C200078350348E50022073367070163F4E6026D
:107C300003A5019178350348E5002CD4220733676A
:107C400007012312E4067CD411C70347040B19C3B0
:107C50002308040A6C483387B7406342E02A03D7FD
:107C60004191231A040663190728035744066854F0
:107C7000B2962A976312D7280317E403634E0726A8
:107C8000639CF526834784050D47850793F7F70F17
:107C9000230CF404637CF7240357A40583570404DE
:107CA000BA97C207C1836374F700231DF4047C5C98
:107CB000639F07367040631A064003D641918327BD
:107CC00009001454138A41916306067EB385F64079
:107CD0001387F5FF634B074605471D8F118F3697B6
:107CE0006345E046B71900209387892FC443139753
:107CF00005014183BE249389892F63D3B7449E2411
:107D0000998FC207C183BA246346B742B305B04016
:107D1000C205C1852685EFE0DFF1DC4083D6C900CE
:107D20000327090023A4F9001C5436971D8F2396BE
:107D3000E90003A7090193D687002320F9005CA37B
:107D400054B393D60701E18374A37CB3832609005F
:107D50001854B387E64063CB0774523493871600F8
:107D6000998F918F6344F0746390E65CB7140020A0
:107D70009387842F83D9C7009C4B9384842FC82773
:107D8000DC37A2075D8DEFD0DFB40D893335A0005D
:107D90004E9542055E3441812310AA0063FDA70879
:107DA0009C48C827DC37A2075D8DEFD09FB20589BC
:107DB00031C19C4883C9D700C827A209B3E9A900EB
:107DC0004165130505FCEFD0FFAF9C48B3F9A9004E
:107DD000C827DC37A2075D8DEFD0BFAF1375E50371
:107DE000EFD05FAE9C4833E5A90042054181C8A7AA
:107DF0002181C8B75E34DEA49C48C827DC37A207BF
:107E00005D8DEFD01FAD098901C5DE24FD17DEA40D
:107E1000CE24C840EFF0AF819C4883D9C400C82766
:107E2000DC37A2075D8DEFD0DFAA0D893335A000C6
:107E3000AA9923103A0183274408638D07329C488E
:107E4000C827DC37A2075D8DEFD0BFA80589631076
:107E50000532832A4408416B130B0BFC03250900F0
:107E600003570A002A9763800A0803A60A014C32C6
:107E70005422A205D58D7422C206D58D7432E20635
:107E8000CD8E83D5CA00B695B305B74063D9053208
:107E9000158F635AE00483274408984B5C335423BE
:107EA000A207D58F898FDEA49C48C827DC37A2079C
:107EB0005D8DEFD01FA2098901C5DE24FD17DEA468
:107EC000CE24C840EFE0BFF69C4883D9C400C82741
:107ED000DC37A2075D8DEFD0DF9F0D893335A00021
:107EE000AA9923103A012322540969A4E391E7DCFB
:107EF0002285EF10F03465BB230C04044DBB3450D5
:107F0000B386D7406342D0128346640213F646001C
:107F100001CAED9A2303D4028356C405231DD40459
:107F20008316C4040356E40442078D86B2962318D0
:107F3000D404835664074183231AE4063697231B2F
:107F4000E40618487CC823090404230C04048D4764
:107F500063F1E7020357A4058356C405835704045D
:107F60006376D702BA97C207C1836374F700231DF3
:107F7000F4048327040885E383270408230E0402FE
:107F800093B71700B307F0407EBC15B3B387F70271
:107F9000B3C7E702C1BF984B48335C2322055D8D10
:107FA0007C23C207C98F683362055D8DEFD09F9532
:107FB00083270408AA8903DAC7009C4BC827DC374B
:107FC000A2075D8DEFD0FF909C400D893335A00056
:107FD0005295B389F9404E95E340A0FA83290408ED
:107FE00083A709002320F4088357440785C383A788
:107FF0000901C827DC37A2075D8DEFD09F8D058969
:1080000011C583574407FD17231AF40603A5490039
:10801000EFE07FE7835784073385A740231CA4063E
:108020004E85EFF08FB4B1B7231A040649B1984BCF
:1080300083A9040048335C2322055D8D7C23C2079D
:10804000C98F683362055D8DEFD0DF8B7C5CAA8AB7
:10805000B389594103DAC7009C4BC827DC37A20714
:108060005D8DEFD01F870D893335A0005295B38900
:10807000A940E3C109C49C403850998FE34CF0C239
:108080008329C40783A709007CDC8357440785C381
:1080900083A70901C827DC37A2075D8DEFD07F8356
:1080A000058911C583574407FD17231AF40603A554
:1080B0004900EFE05FDD835784073385A740231C29
:1080C000A4064E85EFF06FAADDB63C449840998F28
:1080D000E3D507BE8316C40403D7418E420693D569
:1080E00036404182C205C181B307C7408D8FC207A8
:1080F000C18313950701B697C207C187418523162F
:10810000F40463570500198E2E9613150601418558
:108110008316E4048D872322040413D72640338773
:10812000E6402A9742074183BA972317E4042318AD
:10813000F40461B69EA423950400998D8440E1B6B1
:108140003307E04093150701E9B6958FE3D007C0E8
:1081500083476402228593E727002303F402EF108C
:10816000803BEDB61C412322F408EFF00FA003255D
:1081700044086DF983560A005E34032709002285FE
:10818000958F369718D45EB4EFF0EF95DC409A27C0
:1081900009C723A0F19023A204009C48C827DC371C
:1081A000A2075D8DEFD0EFF2058919C59387419045
:1081B00098231367070298A3914A1D4B39AA5C368E
:1081C0004826A2075D8DEFD0CFF0058935C59C48C4
:1081D000C827DC37A2075D8DEFD0AFEF098929ED05
:1081E0009C4883C9D700C827A209B3E9A9005A85CA
:1081F000EFD04FED9C48B3F9A900C827DC37A207A0
:108200005D8DEFD00FED1375E50313651500EFD00D
:108210006FEB33E5A9009C48420541811357850067
:10822000C8A7D8B783D9C400EFD0AFEA0D893335DA
:10823000A000AA9923103A0183A90A005685EFF0FD
:10824000CF92CE8A21B92320F9005C37482783DBFF
:10825000C400A2075D8DEFD0CFE71C540D893335E4
:10826000A0005E953E959C4808D483DBC400C827D7
:10827000DC37A2075D8DEFD0CFE55E340D89333555
:10828000A0005E953385A7404AB42285EFF0AF8504
:10829000CC409E2589CB93870190884335CDEFE074
:1082A0005FC023A204009C48C827DC37A2075D8D6D
:1082B000EFD02FE2058901CD138741901C2393E76E
:1082C00007021CA31C4863945701232864019C40A7
:1082D00026852322F408EFF04F898324440899CCA3
:1082E000984854335C23A206DD8E7C23C207DD8EC2
:1082F0007C33E207D58F1454E387D7F483476402B5
:1083000013F7170001CFF99B93E727002303F4022B
:108310002285EF10402039A08CC361B793E7170086
:108320002303F4026F70DFE92285EF100018832425
:10833000440891E8371500201305852FEFF06F876B
:108340002322A408C5B70327090081491308F7FFB2
:1083500013051700904854325C22A206DD8E7C2261
:10836000C207DD8E7C32E207D58F639CE7023715AA
:1083700000209307852FDA27DE24E3F5E7FA1305BB
:10838000852FEFF00F8359DD638A090023A0A90030
:10839000A685EFF0EFF779B7B6846DBF2322A40866
:1083A000C5BF63900902B306F74063DE06083715C0
:1083B00000201305852FEFE0DFFF2DD52322A40831
:1083C000C1BF83A8090183C5580083C64800A20520
:1083D000D58D83C66800C206D58D83C67800E206B7
:1083E000CD8EB306D84063C00606B306F540634C95
:1083F000D004371500201305852FEFE09FFB2A845A
:1084000015D103A709015C334C23A207DD8D7C2322
:10841000C207CD8F6C3303D7C900E205CD8F83250A
:1084200009003E970D8F635BE0009D8DC20503A59B
:108430004900C1812396B900EFE07F9F23A0890006
:10844000A6852285B9B79440A689B9F6B307F74047
:10845000E35AF0EC5C364826A2075D8DEFD06FC77B
:108460000589E31105EC371500201305852FEFE092
:108470005FF488C0E30805EA98485C334C23A20700
:10848000DD8D7C23C207CD8F6C33DA24E205CD8FDE
:10849000832509003E970D8FE356E0E89D8DC205C8
:1084A000C840C181CEA4EFE09F98ADBD2285EF000A
:1084B000D07F8DBD3387D740634807005A34850786
:1084C000958F998FE350F0E68347640235BDEF72D4
:1084D0003FCE9384019103A904002A848347D900E5
:1084E0000345C900A2075D8DEFD0AFBE31814205C3
:1084F0004181954763FCA7029C405109C827DC379E
:10850000A2075D8DEFD0EFBCB717002003A6872729
:1085100031816D150A054205931506014181C1811E
:10852000814705488948114363E4A7006F709FCADB
:10853000B306F9009822630907016DDB630A17018E
:1085400098326DD7BA9711A08507C207C183E9BFDA
:108550009832E31D67FC13873700E359A7FCB82264
:10856000B4322207558F6363E60011E32E871AA009
:108570009107E1BFEF72DFC04041AA8B1C30082099
:108580004111A2071389C18F5D8DAE892320890017
:10859000EFD02FB48327090019811375C5032A94DE
:1085A00088239C3323A88190A2075D8DEFD06FB202
:1085B0009355650093F5C503B305B0405E85EFE0C4
:1085C0004FE711E503D78B00CD4763E8E7005E85F1
:1085D000EFE00FED41016F707FBE138BC18F03255C
:1085E0000B00CE854105EFD00FFA75F103270B0084
:1085F000370500F01C3B002BA207C18F202B420443
:10860000C18F203B62045D8CEFD0CFAF698C370502
:1086100000E0EFD02FAFE30CA4FA83250B0003D7C3
:108620008B009946138605015E85B105EF10105A3F
:1086300059FD938401919C40C827DC37A2075D8DCA
:10864000EFD02FA93181F155B305B5025E85C20582
:10865000C185EFE00FDE25FD80401C300820A20719
:108660005D8DEFD00FA708A0218108B080403C307D
:108670002820A2075D8DEFD0CFA528A0218128B0AA
:10868000804048305C2022055D8D7C20C207C98F68
:10869000683062055D8DEFD0EFA6935785005CB022
:1086A000935705017CA09357850148A07CB080407A
:1086B00023A4A190938A819008341C2422055D8D07
:1086C0003C24C207C98F283462055D8DEFD08FA38B
:1086D000935785001CB4935705013CA4935785011B
:1086E00008A43CB4804023AAA18E1389418F7C3416
:1086F0006824A2075D8DEFD0CF9D9C4068A42181A6
:1087000068B4C827DC37A2075D8DEFD08F9C137843
:10871000F50F83D88B0093753800B335B000C6953C
:1087200003A3818DC205944003260B009377F803C1
:10873000C181238CF18E239AB1901A840145938CC8
:10874000818F138C419101E403A5018FE9A29C3232
:1087500003CE06005A30A207B3E7C7016312F70E33
:10876000BC3203CE26005A2CA207B3E7C701631917
:10877000F70C58365C2622075D8F7C26C2075D8F7A
:108780007C36E207D98F5840631CF70A183A1C2A36
:1087900022075D8F3C2AC2075D8F3C3AE207D98FE2
:1087A0001840631FF70819C55C4423AC818C5CC575
:1087B0002326640003A74B00B71D0020032684086E
:1087C00093878D2F23A001902382019023A007007F
:1087D0002396170198C723A2770194CB138A41905F
:1087E000138D0190938D8D2F09CE83270409814627
:1087F000A285638A072C084C8297E31A05DC2324A0
:10880000040883C70C0023A6819013F74700938BBD
:10881000C190630D073018488947631AF72A38500A
:1088200083270900631FF72A83470A0093E787001D
:108830002300FA0083476402F99B2303F40255A442
:108840002285404409B798329C2222075D8F5E3111
:108850006392E70C83C83600B822A208B3E8E800A8
:108860005A2D6319170B0343D6008348C600220311
:10887000336313018348E600C20833E3680083488A
:10888000F600E208B3E86800032345006314130907
:10889000034316018348060122033363130183480F
:1088A0002601C20833E3680083483601E208B3E8D2
:1088B000680003230500631F130593764800E398BF
:1088C00006D0937628008DC603A80A001455B30677
:1088D000D84063C606028358C502B386164163407A
:1088E000D0029306C600C295410603250900F1A8EF
:1088F000137818006305080083A7418E1CDDE38808
:1089000005CC8347650293E727002303F502EF00B8
:10891000904075B9484505F903A3018E3E8E1A8A29
:1089200063130A04DC36C826A2075D8DEFC07FFA08
:108930001189E31E05C8944003260B0003550C0063
:108940009C32B83283C8060003C8260083A50A00FB
:10895000A20722079306C600B3E717013367070192
:108960004106AA9559B783280A00638E0800183A71
:108970001C2A22075D8F3C2AC2075D8F3C3AE20722
:10898000D98F639EF812B832BC2222075D8F8357BD
:10899000CA016396E71201C98327CA0023A0418F49
:1089A0005CC523266A00937708019DC39C3283C867
:1089B000060003A80A0003250900A2079306C600C3
:1089C000B3E717014106C2950505EF00D06B01B171
:1089D00013782800E30D08BE03454A01EFE01FF9B4
:1089E0002A84E30605BE83270B000147938607010F
:1089F00099CA943B982BA206D98EB82B4207D98EE0
:108A0000B83B6207558F18C00357CA019386C70049
:108A10005AAC014799CAD437D827A206D98EF8276D
:108A20004207D98EF8376207558F944058C0130516
:108A300004049C329822A207D98F03A70A005EB0D3
:108A40008D471CC8930717001CD41CD8FC36F02691
:108A50007D17A207D18F2312F406231EF404832767
:108A60008A0138D41CCCB717002083D787275EB47F
:108A70007EB483270A021CD083578A0093F7971984
:108A80001EA483A7818D23AC818C5CC4EFF03FA42E
:108A90000355040493054400EFF08F812310A404D0
:108AA00085470147C946014681452285852B11C569
:108AB00081452285EFE0FFE019BE228589BD528500
:108AC000032ACA00B1BD0145EFE07FD43DB383A7BF
:108AD0000A001854998F63C607005A34998FE355DA
:108AE000F0D483470A0013F78700630F073C930510
:108AF000F1002285EFB0DFBA85476316F50018480C
:108B000089476300F71C2285EFC02FA98327C4097A
:108B100081C7084CE9558297A2851385818DEFE0C6
:108B2000DFBCA2850945EFD09FFA61AA898B85C376
:108B30001C480547F917637CF700834764022285C8
:108B400093E727002303F402EF00F01C59BF83A72B
:108B5000418EA308040A130504041CDCEFF03F97C0
:108B60001C481D47F917E36EF7F631678A071307AC
:108B700087BABA979C43828783C70C004947C98B41
:108B80006391E70C83270408984B48335C23220544
:108B90005D8D7C23C207C98F683362055D8DEFC090
:108BA0007FD6832709000505631DF50883576407F1
:108BB00003A70A0094408507231BF40693071700B8
:108BC00068C81CD41CD8FC36F02603550404A20740
:108BD000D18F7D172312F406914738D41CC8930512
:108BE0004400EFE0FFECA947B307F5020357A405E3
:108BF0002310A404231EF40485476315F70006051B
:108C00004205418183578407231DA40403250408DA
:108C1000FD17231CF4061C412320F40891EFFD5797
:108C20007EBCEFE08FF483274409E38807F0084C0B
:108C30000146A285829711B7231F04022309040469
:108C4000CDB783C70C00C18BE38D07E89440035573
:108C50000C0083A50A009C32B83203260B0083C89F
:108C6000060003C82600AA9503250900A2072207CB
:108C70009306C600B3E71701336707014106EF000B
:108C8000904085B583C70C0013F7070169C703251A
:108C9000090078489307F5FF998F63C607083C5091
:108CA000B307F5406341F00891471CC81C508DC7BD
:108CB000084C0146A285829705C185452285EFE0D3
:108CC0005FC003A54D0023A00B00E3050590EFD086
:108CD0003FFD23A20D00FDB822858354A405EFE0DB
:108CE0001FF08357440781C7FD17231AF406054771
:108CF000835704046395E4008607C207C183231DDC
:108D0000F40483470A0093F70702E38C07DC8347E8
:108D10006402228593E727002303F402EF00A07F7B
:108D20009D471CC87DBB944003260B0003580C00D4
:108D30009C32B83203C3060083C8260083A50A000C
:108D4000A20722079306C600B3E76700336717013F
:108D50004106C2952DB7898BE38507D81C5403A71C
:108D60000A00FD17E39FE7D62285EF00B04595BBCB
:108D70002285EFE0DFE671B72285EFE05FE683470B
:108D80000A0093F70702C1C303C70C0083476402BC
:108D9000418B93E727002DC3345003270900639DBF
:108DA000E6042303F4022285EF00E0762285EFE05B
:108DB0000FE583A7818D631DF4005C4423ACF18C27
:108DC000A9471CC803A7018F23A8818E58C411BBD3
:108DD00023A6F18E814689E7E5D623A6018ECDB77D
:108DE000D0476318C40099C223A6F18E5844D8C74F
:108DF000C1BF8546B287C5B72303F4022285EF00C1
:108E00008071A14739BF83C70C00C18BE38B07CCAE
:108E1000385083270900E316F7CC994719B7228504
:108E2000EFE0FFDB83470A0093F70702E38B07CAF3
:108E300083476402228593E727002303F402EF00AF
:108E4000806D2285EFE0AFDB83A7818DE307F4F629
:108E500023A6F18E8146C9D3D047E306C4F88546E0
:108E6000B287D5BF2285EFE09FD783C70C00C18BA7
:108E7000E38907C6385083270900E314F7C6228523
:108E8000EFE0EFD783A7818DE309F4F223A6F18EFB
:108E90008146B9D3D047E308C4F48546B287D5BF2D
:108EA0002285EFE0DFD383C70C00C18BE38B07C2C1
:108EB000385083270900E316F7C283470A0093E777
:108EC00007012300FA0031B9C18B89C72285EFB0B1
:108ED000DFEC99B10356440719C68327C40881C73C
:108EE000084CA285829703260D000DC683C70C008F
:108EF000A18B89C75C3693E717005CB6832704090A
:108F00008146A28595CB084C829709C583270D0021
:108F10002324F40883470A0093F7070289CB8327A9
:108F2000040981460146A28581CF084C829722859B
:108F300023A00B00CD2371B30145EFE05F8DF1B7A6
:108F40000145EFE0DF8CE5B7EF728FA62A894A2D45
:108F500041112E8432C6EFC0FF9608A0218108B0CF
:108F600003554902EFC01F96324628A0218128B040
:108F7000935786000325890250A05CB093570601E1
:108F8000618270B07CA0EFC0BF959357850008A4A4
:108F90001CB4443493570501618128B44824A204C9
:108FA0003CA4C98C4165130505FCEFC0BF91E98C59
:108FB0004145EFC03F91458D4205418148A4218143
:108FC00048B40355E902EFC0FF8F8357E90268A454
:108FD000218168B4231BF9025C344824230904006E
:108FE000A207A30904005D8DEFC0BF8E95671375BE
:108FF000F5035D8DEFC01F8D0357E90283278902BA
:1090000048A4218148B423080400A3080400BA97A7
:109010002328F902228541016F70CF9BEF724F9692
:1090200079712EC63ACA2A89B28A368BBE8D01EE74
:1090300093F73600B3E7FD00595A91C38DC15285AD
:1090400045616F70AF978357650763FAC700834721
:1090500069027D5A93E707F82303F902CDB7939786
:109060002D0013F72D00918BB14611E38146B69781
:109070003EC283270907371D002013074D273EC432
:109080001C475843835489078A07B3D7E702130D57
:109090004D27E3FEF4FA41679306C7FFE3E996FA2A
:1090A00092473082130707FC898393F7F70F9507E0
:1090B00032C85246B207C2073AD2B24C13170B015C
:1090C000C183058A41833ECCD68B8149814732CE0C
:1090D00036D03AD4035A09041247330AEA4063D31C
:1090E0004B015E8A11453ED6131C0A01EFD03F9C0E
:1090F000135C0C012A846306051823200500232233
:10910000050063840914B25788C3F24763810714CA
:10911000C24701460145B305FC00C205C181EFD03D
:109120001FBD48C0630F0514EFD0FFD5B247AA9406
:10913000C204C18081CF5C40E685C843C167FD178A
:109140003376FA0092473E95EF10A03F5C40DC4337
:109150001CC483278D0003274D008A07B3D7E7027D
:1091600063E19712825763EE9710484023168401FB
:10917000D145EFD01FAC631605105C400355C90103
:10918000B38B8B41DC43C20B93DB0B011CC83ED677
:10919000EFC04FF3B25788A3218188B31C48035511
:1091A00049023ED6EFC00FF2B257A8A32181A8B35F
:1091B0001C4822453ED6EFC0AFF2B2571357850088
:1091C000D8B313570501F8A31848C8A36181E8B3C1
:1091D0005C37482723090700A207C98F1255A30946
:1091E00007003ED6EFC00FEEB257E98F22553ED6AC
:1091F000EFC04FEDB2575D8D42051C4841811357BA
:109200008500D8B7C8A72307B401EFC08FEC1C486E
:109210001375F5033ED6E2475D8DEFC0AFEAB25756
:10922000C8A72181C8B7C167FD17337AFA00A247E2
:10923000D29CD2973EC4A287E39E0BE8032AC907BB
:1092400063190A06232E390751A2AA897DBDC2459A
:1092500001460145EFD0BFA948C005C5EFD0BFC248
:10926000AA94C204C180E3860BEEE28505460D4553
:10927000EFD0FFA7AA85484095E1EFD07FA2232237
:109280000400834769027D5A93E707F82303F90234
:10929000E38709DA4E85EFE0EF8F55B323A29501FE
:1092A0008504C20423249401C180EFD09FBF55B52B
:1092B0003E8A83270A00EDFF83270A01835BCA00E9
:1092C000C827DC37A2075D8DEFC0AFE00D893335CD
:1092D000A0005E956305051883270A01C827DC37BF
:1092E000A2075D8DEFC0EFDE0D89631A0516937737
:1092F0003B0081C785476314FB1603D7C90083571A
:10930000CA00BA9703570904634BF7140347EA00EE
:1093100083C7E9006315F71403270A0148335C2368
:1093200022055D8D7C23C207C98F683362055D8D80
:10933000EFC04FDD03A70901835BCA005C23AA9B32
:10934000483322055D8D7C23C207C98F68336205CF
:109350005D8DEFC02FDB6394AB10C247B15503A501
:1093600049009D8DC205C185EFD0BF8CE31B05F080
:1093700003A549003E2599EB1C41FD14C20423A21C
:10938000F90023200500C180EFD09F9193771B0047
:10939000CDC783270A0183CBD700C827A20BB3EB25
:1093A000AB000545EFC00FD283270A0133E5AB00C0
:1093B00042054181C8A72181C8B763958900035C34
:1093C000CA005284CE851145EFD06FF093773B00F1
:1093D00089C7850AC20A93DA0A01137B1B00630856
:1093E0000B008347690293E707022303F9028327EF
:1093F0000907231C9906014AD6972328F9068357A3
:109400006907B38A5741231B5907E30A0CC21C485A
:10941000E38707C25247098BE31307C2C437C82743
:10942000A204C98C2145EFC0EFC91C48458D4205F7
:109430004181C8A72181C8B719B183A54900032577
:109440004A00EFD01FA603D7C9008357CA00BA97B6
:109450002316FA0083A709002320FA00B9BF2320AE
:109460003A01ADB7EF62DFD4AE86814705470146CA
:109470008145EFF0BFBA6F60FFD5AA8708491D4745
:109480006308E5001308E5FF09476155636E0701AE
:10949000014519CAEF62DFD136873E858146814793
:1094A000EFF0DFB76F601FD38280EF62DFCE2A84D8
:1094B0000146D1450545EFD09F8321CD8347640206
:1094C000AA842850F19B2303F402EFC06FC1CC4063
:1094D0002A862285EFF05FA79A2413094400AA89FF
:1094E00099464A86A2852685EF00506E2388A900FA
:1094F0002181A388A9003824343499474A86A2855B
:109500002685EFC0FF842685EFD08FF901456F6077
:10951000DFCB7955EDBF83A7C1906384A736EF6297
:109520003FC6B787002003A70796035AA50523A2C5
:10953000E18A8357450663F347013E8A8347650204
:10954000420A2A84898B135A0A01645D95CB91E4FF
:109550002285EFF09FF56F607FC6984848335C2303
:1095600022055D8D7C23C207C98F683362055D8D3E
:10957000EFC04FB9DE247848998F3E95E36AAAFC84
:109580008329040863960908B71A0020894B938A37
:109590004A27370C0402130B4400FD5CADC0984809
:1095A00048335C2322055D8D7C23C207C98F683355
:1095B00062055D8DEFC00FB5DE247848998F3E952A
:1095C000637CAA048347040B9DEB984848335C23D3
:1095D00022055D8D7C23C207C98F683362055D8DCE
:1095E000EFC04FB2DE247848998F3E9583574406EA
:1095F00063F7A70085472326040A2308F40A834754
:109600006402014593F7F7072303F402A9B7BE8963
:1096100083A70900EDFF8DBF8327040895C3834707
:10962000640213F7470409EF785C01CB144389EA1D
:1096300056270357040463F5E60093F7070AD9D3C6
:109640009C407CDC1C48638977039C4803C9D70095
:10965000C82722093369A9004145EFC0AFA69C483D
:109660003365A90042054181C8A72181C8B7834756
:109670006402F19B2303F402085403A90401EFC020
:109680002FA6935785002304A900A304F90093573C
:1096900005016181A305A9006A342305F90003A926
:1096A0000401EFC02FA27A341C542307A9002181A2
:1096B000A307A900BA977AB81CD8FC24858B99CB4C
:1096C00003A54A0003A904013365AC00EFC04FA114
:1096D000232AA9001C4099E75A85EFC06FA349C50A
:1096E0005C411CC08317E40363949701231F0402A9
:1096F0007C4095E383A7418E98487CC048335C2327
:1097000022055D8D7C23C207C98F683362055D8D9C
:10971000EFC04F9F28C4C84003A90401994658418F
:10972000232225015A863307E940931707013A257A
:10973000C183A2851D8F3AA51A251D8F420741833B
:109740001AA523080900A3080900EF0030482308E0
:10975000A9002181A308A90038243434C8409947BE
:109760005A86A285EFC0CFDE984848335C23220595
:109770005D8D7C23C207C98F683362055D8DEFC0A4
:109780006F989C482A8983DDC400C827DC37A2076C
:109790005D8DEFC00F940D893335A0003C506E9560
:1097A0004A95898F63D3070028D09C4803D9C40009
:1097B000C827DC37A2075D8DEFC0AF910D89333527
:1097C000A0004A955DC98327040823A0040089E707
:1097D00023209408A68999A8984848335C23220539
:1097E0005D8D7C23C207C98F683362055D8DEFC034
:1097F0006F9103A709012A8948335C2322055D8DF7
:109800007C23C207C98F683362055D8DEFC08F8FDF
:109810003305A9406350050613090408832709008E
:1098200081EB832709009CC023209900645CBDB3B1
:10983000984B48335C2322055D8D7C23C207C98F7A
:10984000683362055D8DEFC0EF8B9848AA8D483371
:109850005C2322055D8D7C23C207C98F68336205B6
:109860005D8DEFC02F8A3385AD40E35C05FA032997
:1098700009006DB723A09900B1BF2685EFD0FFAED8
:1098800075B701458280EF621F914111AA8AAE84AB
:10989000B289D14501460545368A3AC63E8BEFD09E
:1098A0000FC56303050E324740412A893A85EFC050
:1098B0006F8108A0218108B05A85EFC0AF8028A031
:1098C000218128B05685EFC0AF819357850048A00D
:1098D0005CB09357050161817CA068B02685EFC01C
:1098E0002F809357850008A41CB444349357050176
:1098F000618128B44824A2043CA4C98C41651305A5
:1099000005FCEFB03FFCE98C5145EFB0BFFB458D46
:1099100042054181B717002048A4218148B403D5EE
:109920008727EFB03FFA68A45C34218168B44824EB
:10993000A207230904005D8DA3090400EFB07FF99D
:1099400095671375F5035D8DEFB0DFF70357890059
:1099500048A4218148B499465286CE852308040044
:10996000A30804004A85EF00702608A8218108B8E2
:1099700099470147930600085286CE854A85EFC075
:109980002FBD4A85EFD0CFB141016F601F8483277F
:10999000050885CBEF62DF813E8714438DE2745D5D
:1099A00014C37CDD834725052320050823220504F5
:1099B00085072309F504EFF01FB66F60BF81368776
:1099C000E9BF8280EF622FFD8324050895C49C4087
:1099D0002A841309C5072320F5088327090099EF76
:1099E000832709009CC02320990083472405232254
:1099F000040485072309F4046F602FFD984B483356
:109A00005C2322055D8D7C23C207C98F6833620504
:109A10005D8DEFB03FEF9848AA8948335C2322055B
:109A20005D8D7C23C207C98F683362055D8DEFB001
:109A30007FED3385A940E35505FA0329090071BF7D
:109A400083270508B1CFEF62AFF6834765022A840A
:109A5000918BA9E7EFF01FF78356A40583574406BF
:109A600013D7160063F4D70013D7170083570404E5
:109A7000231EE404939617006354D700231ED404D6
:109A80000D47B387E7020357C405BA97231DF404B3
:109A90008347640293E747002303F4026F608FF368
:109AA0008280EF624FEFAA840146D1450545EFD091
:109AB0000FA429C52A84A850138944007D15EFB04E
:109AC0003FE24C402A862685EFF00FC81A24AA8967
:109AD00099464A86A6852285EF00500F2388A90063
:109AE0002181A388A900B434994701474A86A685F5
:109AF0002285EFC0EFA52285EFD08F9A6F60EFEC43
:109B0000EF626FE90324050819E0605D5DC41C483D
:109B1000AA84C827DC37A2075D8DEFB09FDB0589DB
:109B200059CD5E24C9EF054AD14501460545EFD020
:109B30000F9C2A8959C118484C41268550335C2313
:109B400022065D8E7C23C207D18F703362065D8E44
:109B5000EFF08FBFAA8963070A0640355C2541658F
:109B60002204130505FC5D8CEFB0DFD5698C4545FB
:109B7000EFB05FD5498C93170401C1832386F900A8
:109B8000A183A386F90003578900138444009946F2
:109B90002286A6854A85EF0070032388A9002181CB
:109BA000A388A900B434994701472286A6854A852F
:109BB000EFC00F9A4A85EFD0AF8E6F600FE1014A78
:109BC000D545A5B718448327490003070700D8AB3C
:109BD0005DBFEF62EFDA404106252A891C3008207C
:109BE0004111A2075D8D2E8AEFB0BFCE21813D8944
:109BF00009050A0563C2A4021C300820A2075D8D76
:109C0000EFB03FCD9355650093F5C503B305B04064
:109C10004A85EFD00F8219C54A85EFD06F88410180
:109C20006F60CFD9832A4900130C0401D285628565
:109C3000EFC06F9583C71A002A8B03C50A00A207DD
:109C40005D8DEFB01FC983C73A00AA8B03C52A00F8
:109C5000A2075D8DEFB0FFC793074004AA86631D7E
:109C6000F506930730046399FB1283270A02638584
:109C70000712C44363820412D44089CE58345C2452
:109C800022075D8F7C24C2075D8F7C34E207D98F69
:109C90006394F61083C77A0003C76A00A207D98FBE
:109CA00099CB03578900C54662869305C4004A854F
:109CB000EF00C07135F1E1554A85EFC09FF729FDEE
:109CC000638C040E9C4CA9DBC84C5E879306C400D1
:109CD0004A86A6858297A1B783A48191014D814DC3
:109CE000938C81911306C07689E463070D0AEA8498
:109CF00055B7BE28639CD708984063150B0439E319
:109D000063160D009C28918B91E3268DDE286392CB
:109D10007709CC4089CD58345C2422075D8F7C24A0
:109D2000C2075D8F7C34E207D98F6394F506E38325
:109D30000DF6DC4423A6FD0083A70C0023A09C00A5
:109D4000DCC489BF1C3883490401A207B3E737018B
:109D500083492401C209B3E7F90083493401E209C8
:109D6000B3E9F900E38EE9F8370500F036C6EFB045
:109D70007FB9B3F9A900370500E0EFB0BFB8B2462C
:109D80001306C076E38EA9F6E31C0BF6A68DC44439
:109D9000A1BFE39DC6FEFDBD18381C2822075D8FBC
:109DA0003C28C2075D8F3C38E207D98F03274A0061
:109DB000E314F7E68144F9BDE3100BE61C380428F0
:109DC000370500F0A207C58F2428C204C58F2438A8
:109DD000E204DD8CEFB01FB3E98C370500E0EFB093
:109DE0007FB2E38BA4E21C300820A2075D8DEFB0A8
:109DF0005FAE93558500BD8989058A054A85EFC008
:109E00005FE38D454A85052301BD83A88191AA861C
:109E10000143C687138881919DE799C998319C2198
:109E200022075D8FBC21C2075D8FBC31E207D98F4D
:109E30009CC225C6B2AA01456316030023A61601DB
:109E40002320D8008280638BD702BA2B6316C70207
:109E500003AE070063140E0055558280F5DD88318E
:109E600098212205598DB8214207598DB8316207D2
:109E7000498F7DD3E302EEFEDC4779BF0543EDBF9A
:109E8000AE2B639AC500050642064182C687DDD324
:109E9000E318E6FED1B7DC47DDBF2167C68705665C
:109EA0007D17F5B7EF622FAF3E292A89AE89B28AB6
:109EB000368B3A8AADC7A1454E85EFC09FD7CE8479
:109EC00001CD0146A1450545EFC07FE2AA847D543E
:109ED00029CDCE85EFC0BFFE03552901C040EFB0AC
:109EE0007F9E08A0218108B05A85EFB0BF9D8327CF
:109EF000090028A0218128B023030400A303040043
:109F0000130B4A0095C703274A004A8B6382E70276
:109F10005D54638C34012685EFC09FD839A001467B
:109F2000AA85EFF09FEE2A8459D522856F60EFA9AC
:109F30008A24EFB03F9948A0218148B083470901A6
:109F4000858B99EB9A24C5465686DA852685BD29E8
:109F50000DC168A0218168B00347A9008346B900FC
:109F60005288C5475686DA852685EFB0DFC82A8431
:109F70004DB7FD577CA07CB0C5B7EF626FA3411110
:109F80002A8432852EC636C432C2EFB07F9819C9F2
:109F9000A2461246B2452A872285EFF0BFF0410162
:109FA0006F604FA37155E5BFEF628FA0562913066E
:109FB0004500EFF09FFC6F60EFA1EF626F9F3E29BD
:109FC0002A84AE843289B1CB814799C898309C20CD
:109FD00022075D8FBC20C2075D8FBC30E207D98F9E
:109FE00018285CC0231A24011367470018A81840DA
:109FF00005EF85CF13054400EFB09F91AA877155F7
:10A0000095C3DC431CC083A68191938781913687D9
:10A0100005E354C480C3014531A00146AA85EFF091
:10A02000DFDE5DD16F600F9BF9FF23200400E1BFED
:10A03000E30387FE5847E9BF0CCD50CD8280EF6225
:10A040002F970545EFC0BFA62A8409C91306000251
:10A050008145EF60EF98930700F83CB422856F606C
:10A060006F97EF624F932A842E8AB289930540023C
:10A0700001460545EFC0BFC729CD03290400404173
:10A08000AA847146CA8523004401A3003401230237
:10A090000400A302040023030400A3030400130527
:10A0A00084004521AE2423010400A301040022857D
:10A0B000112928A0218128B085470147930600086F
:10A0C0001306C90081452685EFB09FC82685EFC0DD
:10A0D0003FBD6F608F8FEF622F8B4041AA8441118B
:10A0E0001C300820AE89A2075D8DEFB08FFE13599A
:10A0F00065001379C903B30A2041C20A93DA0A4101
:10A10000D6852685EFC0FFB239E19E248D4663F0E7
:10A11000F604DC4098236312D704982793868700BF
:10A12000883F3D8B0A0736972C2303483700982F2A
:10A1300022059433598DB82F903BA2054207498FD1
:10A14000A83FB3E505016205598DEFA0DFE4268540
:10A15000EFC01FB541016F60AF86A147E319F7FE5D
:10A160001C38034A0401370500F0A207B3E7470192
:10A17000034A2401014B420AB367FA00034A34013F
:10A18000620A336AFA00EFB0EFF72A8C370500E075
:10A19000EFB04FF7AA8BCE8513050401EFB0BFBE19
:10A1A00019E533758A0133057541333BA000EFA0F3
:10A1B000BFDD51DDE30D0BF89A249D47E3F9E7F885
:10A1C0002685192E49F54209930520022685135943
:10A1D0000941EFC01FA663040512CA852685EFC09A
:10A1E0005FA535F58E2401460945EFC05FB02A8A88
:10A1F00039DDA685EFC0FFCD39F9D6855285032418
:10A200004A00EFC01FA321F52685EFC07FA9D284A5
:10A2100058345C24143822075D8F7C24A20603AADC
:10A220004400C2075D8F7C343D651305F57FE2076E
:10A23000D98F18281CA8D98E38284207D98E3838CB
:10A240006207558F9356870058A454B4935607015C
:10A25000618378B413D7870018B813D70701E18357
:10A2600074A438A83CB8834A3A0083472A002300E4
:10A270000A00A20AB3EAFA00EFB0CFE463E9AA0841
:10A28000056513050580EFB0EFE383473A00034708
:10A290002A00A207D98F85073E95420541812301F7
:10A2A000AA002181A301AA001C340824A2075D8D05
:10A2B000EFB02FE2A1671375F50F5D8DEFB08FE062
:10A2C00008A4218108B4D14523050400A305040096
:10A2D0002285CD2A28A4218128B4CA852685EFC0ED
:10A2E0005F95E31605E64E8885470147930600080B
:10A2F00001469305C4002685EFB0FF8F89BD930505
:10A30000E0FD2685EFC0FF92E30405F089B5056501
:10A3100013050580EFB00FDB83473A0003472A009F
:10A32000A207D98F95BFEF52BFE813F6F50F1105BD
:10A330008D45EFF01FD36F50FFE9EF527FE713F623
:10A34000F50F1105AD45EFF0DFD16F50BFE8EF52CB
:10A350003FE63308B5004208AA86014713580801B2
:10A360008548B307D840C207C18363E4F80493D794
:10A370001500939617003695F956B387D702BE9508
:10A38000C205C18181C51C21A2073E974165930684
:10A39000F5FF93570701758F3385E700C177E98F84
:10A3A00099C3758D050542054181EFB0AFD16F505E
:10A3B0007FE29C3290228906A207D18F13968700F4
:10A3C000A183D18FC207C1833E9761BFEF52DFDB0C
:10A3D000416B41112A89AE8A328ABA84814901448B
:10A3E0007D1B854B631F0908638B09004167931729
:10A3F00084007D172180F98F1374F40F5D8C03C5E1
:10A400001A0083C70A0003470A0022055D8D83C72F
:10A410002A0003463A00C2075D8D83C73A006206F0
:10A42000E207C98F03451A002205498F03452A0018
:10A430004205598D498E41651309F5FF3375260193
:10A44000418233F7270132953A95C1833E952A948C
:10A450003685EFB02FC72A942685EFB0AFC6229578
:10A4600093570501337525013E95935705013375C3
:10A4700025013E951345F5FF4205418141016F508D
:10A480003FD48355A9000325490036C6EFF03FECC1
:10A490002A9493570401337464013E948357A900AE
:10A4A000B246858B89CF931784002180B3893B41C5
:10A4B000B3F767011374F40F93F9F90F5D8C032957
:10A4C00009000DB7EF52DFCEEFF07FE81345F5FF3F
:10A4D000420541816F501FD0EF52FFCBC169AA8462
:10A4E00001490144FD19054A95E0630B09004167E4
:10A4F000931784007D172180F98F1374F40F5D8CFE
:10A500001345F4FF420541816F503FCCAE24C84053
:10A51000EFF0FFE32A9493570401337434013E941F
:10A52000BE24858B89CF93178400218033092A416B
:10A53000B3F737011374F40F1379F90F5D8C84406E
:10A5400065B7B3C7A5008D8B3307C50081E78D477D
:10A5500063EEC700AA876370E50A83C60500850716
:10A560008505A38FD7FEE3EAE7FE82809376350068
:10A57000AA8791CA83C6050085078505A38FD7FEE4
:10A5800093F63700FDB79376C7FF138606FE63F098
:10A59000C70683A3050083A2450083AF850003AFF0
:10A5A000C50083AE050103AE450103A3850183A861
:10A5B000C5019385450223A0770003A8C5FF23A208
:10A5C000570023A4F70123A6E70123A8D70123AA54
:10A5D000C70123AC670023AE17019387470223AE60
:10A5E00007FF75B790419107910523AEC7FEE3EBD6
:10A5F000D7FEE3E4E7F6828039713EDA2ED232D418
:10A6000036D63AD842DC46DE9387818322CC80431B
:10A6100026CA06CEAA8409C41C4C99E32285952338
:10A620000C4454102686228536C6EF00901BF2405B
:10A630006244D2442161828001119387818322CCBC
:10A64000804306CEAA8519C41C4C89E72AC62285F8
:10A650000D2BB245104422856244F24005616F0023
:10A66000907D011126CA4AC806CE22CC4EC652C4DD
:10A67000AA842E8901C51C4D91E321239C4C804462
:10A6800099E32685FD299717000093872756631CB9
:10A69000F402C0408357C400A18BB1C71C48A1C7B6
:10A6A000FD59294A1C4483450900FD17B1E91CC422
:10A6B00063DE07062286A94526854520FD576308E7
:10A6C000F502294535A09717000093872754631496
:10A6D000F4008044C1B7971700009387274FE31B0E
:10A6E000F4FAC04445BFA2852685052A55D97D5573
:10A6F000F2406244D2444249B249224A0561828012
:10A700001CC4050963D70700184C63CBE7006389B5
:10A7100045011C401387170018C02380B70059B7A4
:10A72000228626851D28E31F35F7D1B71C401387E5
:10A73000170018C029472380E70061B793878183FA
:10A74000AA8588436FF0FFF1AA8703C70500850734
:10A750008505A38FE7FE75FB8280011122CC26CAF6
:10A760004AC806CE4EC6AA842E89328401C51C4D25
:10A7700091E3012997170000938747476319F4066F
:10A78000C0401C4C1CC48357C400A18BC9C31C48C7
:10A79000BDCF1C4808409379F90F1379F90F1D8D2F
:10A7A0005C486346F500A2852685652C2DE51C4492
:10A7B0000505FD171CC41C401387170018C0238013
:10A7C00037015C486389A7008357C400858B81CB20
:10A7D000A9476316F900A285268561240DEDF24094
:10A7E00062444A85D2444249B24905618280971742
:10A7F00000009387A7416314F400804459B797176A
:10A8000000009387A73CE31EF4F6C0449DBFA285D9
:10A81000268521203DDD7D59D9B74111938781835C
:10A8200026C2844322C44AC006C62A892E8489C40B
:10A830009C4C99E32685B126971700009387073B28
:10A84000631CF402C0400317C40093170701C183BF
:10A8500093F68700B5EE93F607019DEEA5472320FA
:10A86000F900136707042316E4007D55B240224423
:10A87000924402494101828097170000938707396B
:10A880006314F4008044C1B797170000938707341E
:10A89000E31BF4FAC04445BF918B8DC74C5889C95E
:10A8A000930744046384F5004A85A923232A0402FC
:10A8B0008357C4002322040093F7B7FD2316F40046
:10A8C0001C481CC08357C40093E787002316F4007C
:10A8D0001C4881EF8357C4001307002093F7072813
:10A8E0006385E700A2854A85B5218357C40013F725
:10A8F000170005C75C4823240400B307F0401CCCB4
:10A900001C480145A5F78317C40013F7070839DF72
:10A9100093E707042316F40089BF898B014791E36D
:10A92000584818C4F1BF83D7C500011122CC26CAEC
:10A9300006CE4AC84EC613F78700AA842E8471EF4C
:10A94000D841634DE000B841634AE0000145F24060
:10A950006244D2444249B2490561828058547DD74D
:10A9600003A904009396370123A0040063DD0606C3
:10A9700070488357C400918B99C75C401D8E5C580A
:10A9800099C33C401D8E5C540C50814626858297AD
:10A99000FD570357C400631DF5009440F54763E875
:10A9A000D706B70740208507B3D7D700858BA5C347
:10A9B0001C48232204001CC09317370163D80700EA
:10A9C000FD576314F5009C4091E368C84C5823A0E0
:10A9D0002401ADDD930744046384F500268519291D
:10A9E000232A0402A5B70C50014685462685029706
:10A9F000FD572A86E31FF5F69C40A5DF7547638562
:10AA0000E70059476394E70423A0240181B7136743
:10AA100007042316E4007D551DBF83A90501E387C4
:10AA200009F203A905008D8B23A0350133093941B3
:10AA3000014791E3D84918C4E35A20F11C540C5043
:10AA4000CA864E86268582976349A0008357C40034
:10AA500093E707042316F4007DBFAA993309A940A0
:10AA6000E1BF9C49A5C3011122CC06CE2A8411C5A1
:10AA70001C4D81E72EC63122B245971700009387FF
:10AA8000E716639CF5004C408397C5009DC722855F
:10AA90006244F24005616FF01FE997170000938749
:10AAA000E7166394F5000C44C5B797170000938729
:10AAB000E711E39BF5FC4C44C1BFF2406244014501
:10AAC0000561828001458280411122C406C62A8424
:10AAD0002316B5002317C5002320050023220500F7
:10AAE000232405002322050623280500232A050028
:10AAF000232C0500214681451305C505EF504FEE77
:10AB0000971700009387E7BE5CD0971700009387E4
:10AB100047C11CD497170000938787C55CD497174B
:10AB20000000938747C800D01CD8B240224441019E
:10AB3000828097050000938505F391AA411126C2F2
:10AB4000130680069384F5FFB384C4024AC02E899D
:10AB500022C406C69385440791262A8401CD23206A
:10AB6000050023222501310508C41386840681458A
:10AB7000EF500FE72285B24022449244024941013E
:10AB800082801C4DA5E7411106C622C4970700002C
:10AB9000938767FA1CD59387C1859C4323240504BA
:10ABA00023260504232805046314F50085471CCDDE
:10ABB0002A84352848C022851D2808C422850528F6
:10ABC00048C4484001469145EFF01FF0084405464F
:10ABD000A545EFF07FEF48440946C945EFF0DFEEA9
:10ABE00085471CCCB24022444101828082804111C1
:10ABF0009387C18526C284434AC006C69C4C22C4A2
:10AC00002A8981E72685EFF0DFF793848404804466
:10AC1000DC40FD1763D607009C40B9CF8440C5BF18
:10AC20000317C40039E7C1778507232204062320D0
:10AC3000040023220400232404005CC4232804000D
:10AC4000232A0400232C0400214681451305C40552
:10AC5000EF500FD9232A0402232C040223240404D6
:10AC6000232604042285B240224492440249410131
:10AC700082801304840671BF91454A85EFF01FEC72
:10AC800088C049FDB1472320F9000144E1BF797133
:10AC900022D44AD052CC56CA5AC85EC606D626D24C
:10ACA0004ECE2A8AAE8A130485040149054BFD5B0A
:10ACB00009ECB25022544A8592540259F249624A30
:10ACC000D24A424BB24B45618280044483294400FE
:10ACD000FD1963D409000040E1BF83D7C400637B42
:10ACE000FB008397E40063877701A6855285829AEB
:10ACF0003369A90093848406E1BF1971A6DAAE8492
:10AD00008395E500A2DC86DE328463DC050083D710
:10AD1000C40023A0060093F7070885E793070040C7
:10AD20001DA0300836C6EF00902EB246E34105FE66
:10AD30007247BD67F98F7977BA9793B717009CC2AE
:10AD4000F1BF930700041CC0F6506654D654014569
:10AD50000961828083D7C500011122CC06CE26CAA4
:10AD60004AC8898B2E8489CF930774041CC01CC8E1
:10AD700085475CC8F2406244D24442490561828002
:10AD800074003000AA84EFF05FF7A2452A89268577
:10AD9000312201ED8317C40013F7072061FFF19BF7
:10ADA00093E727002316F400C1B7970700009387A5
:10ADB00087D89CD48357C40008C008C893E7070805
:10ADC0002316F400A2475CC8B24791CF8315E40074
:10ADD0002685EF00F02601C98357C400F19B93E755
:10ADE00017002316F4008357C4003369F9002316B3
:10ADF000240149B7DDC183A7C5FF411122C406C69E
:10AE000026C21384C5FF63D307003E94AA84EF00D3
:10AE1000102B9387C1919C4381EF2322040023AE22
:10AE200081902244B2402685924441016F0050290E
:10AE3000637EF40014403307D4006396E700984320
:10AE4000DC43369718C05CC0D9BFBA87D84319C352
:10AE5000E37DE4FE94433386D700631F86001040F1
:10AE6000B29694C33386D700E31DC7FA1043584304
:10AE7000B29694C3D8C375B76375C400B1479CC07C
:10AE80004DB71040B306C4006316D70014435843AF
:10AE9000B29614C058C0C0C369B78280011126CAD7
:10AEA00093843500F19806CE22CC4AC84EC6A10440
:10AEB000B14763F5F404B14463E4B4042A89EF00B4
:10AEC00010209387C19198433A8429E49387019293
:10AED0009C4399E781454A85EF00407E23A0A192DB
:10AEE000A6854A85EF00807DFD5963193507B14776
:10AEF0002320F9004A85EF00B01C29A0E3DE04FA04
:10AF0000B1471CC10145F2406244D2444249B249B2
:10AF1000056182801C40858F63CF0702AD4663F6D2
:10AF2000F6001CC03E9404C031A05C40631387024D
:10AF300023AEF1904A85EF00B0181305B4009307D3
:10AF4000440061993307F5405DDF3A94898F1CC056
:10AF50005DBF5CC3C5B72287404085BF1304350081
:10AF60007198E30285FCB305A4404A85812FE31C58
:10AF700035FBB5BF1C46FD171CC663DA0700184E2B
:10AF800063C5E700A9476394F5006FF00FFD1C420D
:10AF90002E851387170018C22380B7008280011105
:10AFA00022CC26CA4AC84EC652C406CE2A89AE89C9
:10AFB0003284B304D6007D5A63149400014511A86D
:10AFC000834504004E864A85EFF0DFFA0504E31559
:10AFD00045FFF2406244D2444249B249224A0561E7
:10AFE0008280357122CD26CB4AC94EC706CF52C5C5
:10AFF00056C35AC1DEDEE2DCE6DAAA89AE843289C3
:10B00000368409C51C4D99E3EFF0BFB797170000D0
:10B010009387C7BD639DF40C83A4490083D7C40004
:10B02000A18BE5CB9C48F5C793070002A304F1026E
:10B030009307000302D22305F10222C6930B5002AC
:10B04000971A0000938A8ABE054C294B4A8483478D
:10B05000040099C36392770FB30C2441638E0C00F4
:10B06000E6864A86A6854E85EFF07FF3FD57630797
:10B07000F51E9256E69636D2834704006380071E7B
:10B08000FD571309140002C802CE3ECA02CCA30920
:10B09000010482D48345090015465685EF009000CF
:10B0A00013041900C24759E913F7070109C7130729
:10B0B0000002A309E10413F7870009C71307B002D0
:10B0C000A309E104834609001307A0026380E60890
:10B0D000F2474A848146254603470400930514003D
:10B0E000130707FD6379E60AB5CA3ECE85A8971710
:10B0F00000009387A7B16395F40083A4890039BF4A
:10B1000097170000938787ACE39AF4F083A4C900F3
:10B1100031B7A6854E85EFF04FF019D57D55FA4031
:10B120006A44DA444A49BA492A4A9A4A0A4BF65BBF
:10B13000665CD65C0D618280050411BF3305554104
:10B140003315AC00C98F3EC82289A9B73247930690
:10B150004700184336C6634907023ACE0347040046
:10B160009307E002631FF704034714009307A0024C
:10B17000631BF702B2470904138747009C433AC692
:10B1800063C107023ECA35A83307E04093E72700B2
:10B190003ACE3EC8E1B7B387670385462E84BA9797
:10B1A00025BFFD57C5B7050402CA8146814725461C
:10B1B0000347040093051400130707FD6376E606B2
:10B1C000F1F2834504000D4617150000130585A60E
:10B1D000D12D11CD971700009387C7A51D8D93071B
:10B1E0000004B397A700424505045D8D2AC8834536
:10B1F0000400194617150000130505A413091400CF
:10B200002304B10245253DC19757FFFF938787DF90
:10B2100095E74247B2471377071009CF91073EC61B
:10B220009257D2973ED21DB5B387670385462E84C9
:10B23000BA97BDBF9D07E19BA107D5B778009706D8
:10B240000000938606D626860C084E8597000000DF
:10B25000E7000000FD572A8AE314F5FC83D7C400F9
:10B2600093F70704E39C07EA125555BD780097064B
:10B270000000938606D326860C084E85012AD9BF86
:10B28000797156CA9C49BA8A984522D426D24ECEA4
:10B2900052CC06D64AD05AC85EC6AA892E84B28439
:10B2A000368A63D3E700BA879CC00347340419C3C6
:10B2B00085079CC01C4093F7070281C79C40890703
:10B2C0009CC00329040013796900631A0900130B59
:10B2D0009401FD5B5C449840998F634CF9041C40D9
:10B2E0008346340493F70702B336D000A5EB130668
:10B2F0003404D2854E85829AFD576303F5041C40C1
:10B3000011469840998B544481446397C700B38495
:10B31000E64063D3040081441C4418486354F7009A
:10B32000998FBE94014969047D5B639824050145AA
:10B3300009A885465A86D2854E85829A631E750174
:10B340007D55B250225492540259F249624AD24A6F
:10B35000424BB24B456182800509ADBF3307D40033
:10B3600013060003A301C704034754049387160080
:10B37000A2978906A381E7049DBF85462286D285D0
:10B380004E85829AE30E65FB050945B7797122D493
:10B3900026D24AD04ECE06D652CC56CA5AC8B68904
:10B3A00083C68501930790063289AA842E8413866A
:10B3B0003504638DF60263E2D70693078005638840
:10B3C000F61863EDD7006381062293073004638E7D
:10B3D000F60A930A24042301D404C9A09307300673
:10B3E0006385F60A93074006E395F6FE1C40084382
:10B3F00093F6070893054500C5C61C410CC363D8E6
:10B4000007001307D002B307F040A301E404971626
:10B4100000009386E68229476DA89307000763849E
:10B42000F61663E5D7029307E006638BF6189307D9
:10B43000F006E390F6FA0C401C4313F80508138558
:10B4400047006307080608C39C438DA8930750076D
:10B45000E383F6FE93078007638BF61293073007AA
:10B46000E399F6F61C43D04181459386470014C307
:10B4700083AA070056853D2101C53305554148C0C3
:10B480005C401CC8A301040471A81C43930A240453
:10B49000938647009C4314C32301F4048547D5B722
:10B4A00093F607041C410CC3B9DAC207C18781BFF8
:10B4B00093F5050408C3C9D983D707001307F0061D
:10B4C0006388E60E97060000938686772947A301D6
:10B4D00004044C400CC463C5050008406D9908C0C5
:10B4E00099E3B28A91CDB28AB3F5E702FD1AB69517
:10B4F00083C505002380BA00B3D5E70263F0E70CEB
:10B50000A147631EF7001C40858B91CB58401C4817
:10B5100063C7E70093070003A38FFAFEFD1A330603
:10B52000564110C84E87CA867000A2852685EFF066
:10B530003FD57D5A631E450B7D55B250225492541F
:10B540000259F249624AD24A424B45618280A38243
:10B55000D504970600009386A66E0C40084313F8A6
:10B5600005081C411105630D080208C313F71500F7
:10B5700001C793E505020CC04147B1FB0C4093F5B0
:10B58000F5FD0CC0A9B79C4193E707029CC1930746
:10B590008007A302F404970600009386A66B75BF8C
:10B5A00013F8050408C3E30308FCC207C1837DBF89
:10B5B000970600009386C668214711BFAE872DB756
:10B5C00094411C43CC4913F80608138547006306D1
:10B5D000080008C39C438CC301A808C393F6060463
:10B5E0009C43F5DA2390B70023280400B28A1DBFDC
:10B5F00014485686CA8526858299E30F45F31C4078
:10B60000898B8DE7B2474844E359F5F23E8535B75B
:10B6100085465686CA8526858299E30F65F1050A17
:10B620005C443247998FE345FAFEE9BF014A930A29
:10B6300094017D5BF5B7011122CC06CE2A8409C99D
:10B640001C4D99E732C62EC4EFF0AFD33246A24567
:10B6500097070000938787596316F60250401C46EF
:10B66000FD171CC663D00704184E63C7E70093F7A5
:10B67000F50F29476398E70222856244F24005618D
:10B680006FF0AF8D97070000938747586314F6005B
:10B690001044F1B79707000093874753E311F6FC76
:10B6A000504475BF1C4213F5F50F1387170018C2DD
:10B6B0002380B700F240624405618280411122C4B8
:10B6C0002A842E8597D7FF1F23A607E006C6EF80A2
:10B6D000CF94FD576319F50097D7FF1F938787DF36
:10B6E0009C4391C31CC0B24022444101828041115D
:10B6F00022C42E848395E50006C6E1226349050035
:10B700007C48AA977CC8B24022444101828083577A
:10B71000C4007D777D17F98F2316F400EDB783D72A
:10B72000C500011122CC26CA4AC84EC606CE93F7E0
:10B730000710AA842E843289B68991C78395E500C3
:10B740008946014635228357C4007D777D17F98FDE
:10B750002316F4008315E4006244F240CE864A8644
:10B76000B24942492685D24405613DA8411122C40F
:10B770002E848395E50006C6E528FD570357C400CF
:10B78000631BF500FD77FD17F98F2316F400B24017
:10B790002244410182808567D98F2316F40068C84E
:10B7A000FDB78395E50025A8411122C42A842E8582
:10B7B000B285368697D7FF1F23AE07D006C6EF8027
:10B7C0000F81FD576319F50097D7FF1F938787D027
:10B7D0009C4391C31CC0B24022444101828041116C
:10B7E00022C42A842E8597D7FF1F23A507CE06C61D
:10B7F0001922FD576319F50097D7FF1F938787CD4F
:10B800009C4391C31CC0B24022444101828041113B
:10B8100022C42A842E85B28597D7FF1F23AC07CA7E
:10B8200006C6D520FD576319F50097D7FF1F9387EC
:10B8300067CA9C4391C31CC0B2402244410182802C
:10B84000411122C42A842E8597D7FF1F23A407C83D
:10B8500006C6D120FD576319F50097D7FF1F9387C0
:10B8600067C79C4391C31CC0B240224441018280FF
:10B87000411122C42A842E85B285368697D7FF1FB0
:10B8800023AA07C406C64520FD576319F50097D7BC
:10B89000FF1F938727C49C4391C31CC0B24022441E
:10B8A0004101828093F5F50F2A966314C500014586
:10B8B000828083470500E38DB7FE0505FDB78280D2
:10B8C0008280411122C42A842E85B285368697D77C
:10B8D000FF1F23A107C006C6B928FD576319F5004D
:10B8E00097D7FF1F938707BF9C4391C31CC0B240EB
:10B8F0002244410182809307800517D7FF1F232B25
:10B90000F7BC7D5582809307800517D7FF1F23233F
:10B91000F7BC7D5582809307800517D7FF1F232B27
:10B92000F7BA014582809307800517D7FF1F2323AD
:10B93000F7BA7D5582809307800517D7FF1F232B09
:10B94000F7B87D5582800000486172644661756C6D
:10B95000745F48616E646C65720D00006D636175A3
:10B9600073653A253038780D0A0000006D747661F1
:10B970006C3A253038780D0A000000006D65706360
:10B980003A253038780D0A00536F636B657449644B
:10B99000466F724C697374656E2025640D0A000051
:10B9A00047494E545F535441545F554E52454143AD
:10B9B000480D000047494E545F535441545F49506D
:10B9C0005F434F4E464C490D00000000504859203F
:10B9D0004C696E6B20537563636573730D000000D3
:10B9E00054435020436F6E6E6563742053756363D8
:10B9F0006573730D00000000736F636B65742069DD
:10BA0000643A2025640D0A0054435020446973634E
:10BA10006F6E6E6563740D005443502054696D65FC
:10BA20006F75740D000000004572726F723A202528
:10BA30003032580D0A000000546370536572766509
:10BA40007220546573740D0053797374656D436C83
:10BA50006B3A25640D0A00006E657420766572737A
:10BA6000696F6E3A25780A0076657273696F6E2089
:10BA70006572726F722E00006D6163206164647282
:10BA80003A000000257820005743484E45545F4C4B
:10BA90006962496E697420537563636573730D0041
:10BAA000380900000A0A0000480A00001E0B0000C6
:10BAB000820F0000BC0F00004A180000EE1B0000BF
:10BAC0006C1B0000660B0000780B0000EE1B0000F2
:10BAD000EE1B0000EE1B0000EE1B0000EE1B000042
:10BAE0009A0B00001C0D00007C0D0000A20D000050
:10BAF0006C0E0000D00E00002E0F0000EE1B0000A8
:10BB0000EE1B0000EE1B0000EE1B0000EE1B000011
:10BB1000EE1B0000C80D0000574946492044415023
:10BB2000000000005749464920434D5349532D44D6
:10BB30004150207632000000303132333435363710
:10BB400038390000322E30000000000001000100F2
:10BB500002000400030004001C002000B4002400C4
:10BB6000140010001000FC05001112131415161714
:10BB700018191A1B1C1D1E1F78770000BE770000C5
:10BB8000D8770000E8770000E8770000D47700005D
:10BB9000D4770000F67700000102030405060707CA
:10BBA0000707070707000000788B0000848C00005F
:10BBB000708D0000788D00001E8E0000708D0000DA
:10BBC000648E0000A08E0000000000000000000055
:10BBD0000000000000000000000000000000000065
:10BBE0000000000000000000000000000000000055
:10BBF0000000000000000000000000000000000045
:10BC00000000000000000000000000000000000034
:10BC10000000000000000000000000000000000024
:10BC20000000000000000000232D302B2000000049
:10BC3000686C4C006566674546470000303132331A
:10BC40003435363738394142434445460000000018
:10BC50003031323334353637383961626364656682
:04BC600000000000E0
:10BC6400000000000102030401020304060708099E
:10BC740000000000E8BB000008BC0000C8BB0000D6
:10BC840000000000000000000000000000000000B0
:10BC940000000000000000000000000000000000A0
:10BCA4000000000000000000000000000000000090
:10BCB4000000000000000000000000000000000080
:10BCC4000000000000000000000000000000000070
:10BCD40000140140C0A80101C0A8010AFFFFFF0031
:10BCE400A80C0000000E2707D484002002040608D4
:10BCF400A87F00200000CDAB48BB000058BB00006B
:10BD04006E1900000010000010000020FFFFFFFF6C
:10BD1400FFFF000000000000000000000000000021
:10BD2400FFFFFFFF03060C183060780010000020AE
:00000001FF
